:10000000F01F0010655000006350000063500000B6
:1000100063500000635000006350000000000000C7
:10002000000000000000000000000000635000001D
:10003000635000000000000063500000092200002F
:1000400011200000112000001120000011200000EC
:1000500011200000112000001120000011200000DC
:1000600011200000112000001120000011200000CC
:10007000112000006150000061500000C10000002C
:10008000D1220000E9220000FD2400001525000017
:1000900061500000592600006150000061500000CE
:1000A000615000006150000061500000615000008C
:1000B000615000006150000061500000615000007C
:1000C000554B10B51A6801321A60544B1A68544BDC
:1000D000D2B2302A69D01ADC182A44D012DC082A9D
:1000E00032D0102A00D094E04E4A002111604E49CF
:1000F0000A68501C08604D49895C4D4AC9B21160BC
:10010000282287E0202A63D0282A32D081E0482A9A
:100110005ED004DC382A51D0402A53D079E0502AEE
:1001200060D0582A75D13F490A68501C0860404980
:1001300008684049C0B288543F4A0221FF3111602B
:1001400080221021D20563E0374A00211160116836
:10015000481C1060354A515C354AC9B211602822EA
:100160001A6001223CE030490A68501C08602F499F
:1001700009E02D4A314910680968884207D21168A0
:10018000481C1060294A515C294AC9B240E02C4AF7
:1001900011688022D205002901D0202138E02649AB
:1001A0000220FF300860102132E08022D2051021A9
:1001B000116008221A608122520011E08221490058
:1001C0001D4A25E01E4A1168042201291AD11DE0AA
:1001D0008022D2051021116008221A600422FF3209
:1001E000154B17E00F4A1168481C1060104804684E
:1001F0001048E4B244541068114A116804220139CD
:10020000884203D28021C9050A6002E01A6000E03A
:10021000116008221A6010BD88020010040000401E
:10022000180000407C02001084020010AC04001092
:10023000080000409C04001080020010BC04001064
:10024000980400101B4B02211A6810B50A431A606B
:10025000194B20211A68041C0A431A60174B1849CD
:100260001A680A401A601868012210431860154B7A
:1002700018680140196019680A431A60124B6C2211
:100280001A60124B1249186804F072FF114A10608C
:10029000114A1060022C02D1104BA0221A60104BA0
:1002A000802212021A6080234022DB0501201A609E
:1002B00010BDC046048004408080044030400440AB
:1002C000F8FCFFFF34400440180000409004001088
:1002D000400D030014000040100000400C000040DE
:1002E00000E100E0034B1B689A06FBD5024B186047
:1002F0007047C0461480004000800040FFFFFFFFB1
:1003000070B5061C00200D1C01F072F9002801D008
:1003100002F078FD00242C60301C3460291C01F0B0
:1003200095F9201C01F064F9A04207D002F06AFDA3
:100330002C60301C3460291C01F088F970BD08B5B0
:1003400001F092FF08BD08B500230B60036001F0C7
:100350007DF908BD10B502F01DFD0D4B0020196898
:1003600002F042F9002002F02FF9002002F00CF90F
:10037000084B01241C60084B201C198801F0F0FF79
:10038000201C01F0DDFF201C01F0BAFF10BDC046AB
:100390008C040010780200109404001037B50C246F
:1003A0000120032101F02CFF684601A9FFF7A8FFF7
:1003B000009D002D02D1013C002CF1D1FFF7CAFFB6
:1003C000281C3EBD08B5002002F0EEF8012001F027
:1003D000A7FF02F0E5FC08BD38B5051C0C1CFFF7B3
:1003E000B9FF054B0122281C211C5A6204F03EF87B
:1003F000FFF7E8FF38BDC046680C001010B5041CBC
:10040000FFF7A8FF201C03F0A1FF041CFFF7DAFF91
:10041000201C10BD08B50020FFF7F0FF08BD00004C
:1004200008B5021C0249034802F03CFB08BDC04667
:10043000A05200009852000037B500F04FFF032291
:10044000164B1748002101F037F800F051FFFFF775
:10045000E1FF1448FFF7E4FF134B144A00241A602D
:100460001D1C2B689C4211DA02F0D8F9002803D039
:1004700001F0A6FC00240FE00A2001F0F5FE68461A
:1004800001A9FFF73DFF009B002B05D0FFF7C2FF3E
:10049000074802F007FB37BD0134E2E7C85B000004
:1004A000A9520000B85200007C0300107017000031
:1004B000BE520000704700001B4B73B5041C1B4963
:1004C000186804F055FE1A4900901A4A1A4B201C6D
:1004D00002F0F4FA01F096F9002812D001F0AEF91A
:1004E000FA218900061C04F043FE051C201C02F0C2
:1004F00036FB124B20186B431149F3182A1C02F0EB
:10050000DDFA201C02F02BFB0E4B20181B68002B81
:1005100002D003DA0C4A02E00C4A00E00C4A0D4912
:1005200002F0CCFA73BDC0469004001040420F00A8
:10053000CF520000A0520000DC52000018FCFFFF68
:10054000E052000048010010CC520000C9520000E7
:10055000999B0000EB52000070B5051C0E1C141C8A
:1005600000F0BCFE301C291C0022064B00F0A4FF4A
:10057000201C01210922044B00F09EFF00F0B8FE70
:1005800070BDC046C85B0000C05B000000B5084BF2
:1005900089B01A78074B68461B78074902F08EFA33
:1005A00001206946054AFFF7D7FF09B000BDC046E4
:1005B0003C010010000000101F5300002D530000EC
:1005C000F0B52A4C2A4D237885B001932F78FFF798
:1005D000DDFFFFF71FFF002602A803A9FFF790FE2B
:1005E000029800282BD0C0B200F080FF40280CD029
:1005F00004D830280ED0392817D01BE0462830D038
:1006000049280DD0412815D126E02B783E2B11D852
:10061000013303E02B78002B0CD0013B2B7009E059
:100620002378062B06D8013303E02378002B01D072
:10063000013B237000F03EFEFFF7A8FF0026029B5F
:10064000002B02D0C82001F00FFE04200321013648
:1006500001F0D6FD1D2EBFDD019B2F70237000F031
:1006600029FEFFF7D7FE05B0F0BDC0460000001020
:100670003C01001038B5051C0C1C00F0FAFD291CCB
:10068000221C0120FFF768FF034B00225A60034A37
:10069000943212689A6038BD680C0010CC040010C7
:1006A00010B590B0041C6846FFF706FF201C694691
:1006B0006A46FFF751FF10B010BD000000B52D22B3
:1006C0008DB0002800D02B2268460D4902F0F6F9C3
:1006D00004A802F029FC0120694604AAFFF73CFFA8
:1006E0000320002101F08CFD0220FFF787FE002887
:1006F000EED00A20002101F083FD0DB000BDC04600
:100700006053000070B58CB0FFF784FE02A8144956
:1007100002F02EFA2E25FF3504AE301C02F004FC48
:100720006846002409A90930F47402F021FA02AAEB
:100730000420311CFFF710FF201C032101F060FD95
:10074000684601A901940094FFF7DAFD009BA342DB
:1007500002D1013DA542DFD1FFF75CFE0CB070BDB8
:100760009A9B0000F0B5002493B00594FFF752FE69
:100770000222962301940392251C5B00029300F051
:10078000ADFD019B9A4F002B6DD10AAE301C02F0DB
:10079000CBFB019AF27432747273B272F2713271DD
:1007A000002C01D1012D05D1301C042100223B1C5D
:1007B00000F082FE8F4E3B1C301C1E21002200F0F8
:1007C0007BFE8B4F012C01D1012D06D168462D30C7
:1007D000252100223B1C00F06FFE301C332100223B
:1007E0003B1C00F069FE824E022C09D1012D07D07E
:1007F000684633304D210022331C00F05DFE09E0D5
:100800000CA83A210022331C00F056FE032CEFD135
:10081000012DEDD0784F331C381C5921002200F0F7
:100820004BFE734E042C01D1012D06D168463630A3
:100830005F210022331C00F03FFE381C6C21002297
:10084000331C00F039FE052C01D1012D06D168467C
:10085000393072210022664B00F02EFE0FA80421D1
:100860000922664B03E06648042100223B1C00F08D
:1008700023FE00F03DFD059B002B0AD0143B012B0D
:1008800005D8052C03D0962001F0EEFC01E0FFF71F
:10089000C1FD0320011C01F0B3FC5A4B1E68002E61
:1008A000F7D1301C00F0A4FE06A9071C05A8069687
:1008B0000596FFF725FD059B002B73D007AE08AF0B
:1008C000301C391C09AA02F063FB019000286FD18B
:1008D000301C02F047FC051C05981238052866D824
:1008E00004F0E4FB0565240C6503601C00E0601D5A
:1008F000062104F093FC00250C1C59E0052C56D869
:10090000201C04F0D3FB03060B0D10393388013390
:1009100016E0B0780C2104F021FC18E001355DE010
:10092000387801301AE0787801301FE0052C3ED885
:10093000201C04F0BBFB03070F1119213388013B76
:10094000338044E0B0780C210A3004F067FC0131B8
:10095000B1703CE0013D41E038781730182104F0D7
:100960005DFC042239703FE078783B303C2104F094
:1009700055FC032379702FE00023BB70281C07214E
:1009800004F04CFC301C0A1C0991391C052C02D1C6
:1009900002F059FB02E0039B02F014FB01259623B1
:1009A000AB4007E0002F06D101235D4003E00125A5
:1009B00096235B000293059B842B17D0182B15D030
:1009C000029B029A013B002A00D0D7E60EE0301CC1
:1009D00002F0C8FB0523051C0393CFE7281C311C3C
:1009E00002F0F0FB022405220392C7E713B0F0BD2A
:1009F000C85B0000695300005E530000C05B00004C
:100A00006B53000060020010F7B502F023FA1820C3
:100A10000021FFF7E1FC0024694EFFF7D3FC694D8C
:100A200000236B62201C02F036FA002C02D000205A
:100A3000012101E00620032101F0E2FB201C02F06D
:100A400025FA01A9071C6846002F03D0FFF77BFC9D
:100A5000012723E0FFF777FC009A002A1ED1002C23
:100A6000E0D1594B1B68002BDCD1584B98331B68E5
:100A7000002B05D1564BF618D4D5182300931DE052
:100A8000544B00941A6811321A60009A102AF1DC53
:100A900003F00CFC009B01330093F6E7002C0DD013
:100AA000009B182B02D00124002FB6D000F028FCA8
:100AB0004948FFF7B5FC454B0122DA6600F0D0FE4D
:100AC00002F032F9009A182A62D1019F0024F8B28C
:100AD00000F00CFD012601946E62172846D00CD858
:100AE00013282BD002D8112819D04EE015282DD06C
:100AF00016284AD1FFF764FD4AE026282ED004D8F4
:100B000019281ED0212811D03FE0442836D045288E
:100B10003BD1E120000102F0AFFA301C32E02F4B54
:100B20001B68002B34D0FFF7EDFD05E02B4B1B6855
:100B3000002B2DD0FFF716FE009429E0FFF77CFC78
:100B400026E0274B1868301A00F0B0FF0120FFF7AD
:100B5000A7FDFFF75FFCFFF721FC19E0214B052201
:100B60001C70214B1A7000F0A5FB11E01F4B1A6896
:100B700001321A60052A0BD11C6009E01C4802F002
:100B80007BFA201CFFF79AFD02E0002301976B62BD
:100B9000FFF7E0FB0098019903F068FC6B6A002BFB
:100BA00001D0FFF737FC094B94331B68002B03D1AE
:100BB00000F048FB01242FE704F0F2F92BE7C046D0
:100BC00020BF0200680C001060020010CC0400106E
:100BD0000CFEFFFF8C02001079530000480100104A
:100BE000080000103C01001000000010140100106B
:100BF000F0F1FFFF73B501F0F9FF3A4C00F0BAFCD9
:100C00003948002101F074F90021384801F070F9E9
:100C100000F088FD00F028FF23680726B343236017
:100C2000236801252B4300202360021C0B2101F0C7
:100C3000E9F8201C2E4C102101F05AF923680022FB
:100C4000B34323602368281C2360042101F0DAF8F1
:100C5000201C002101F04CF901F0BEF896200002A2
:100C600001F038FD234D01235B4200202B60FFF78C
:100C700017FD00232B6050240120FFF7E3FA00F05A
:100C8000F3FE02F0B1F82B68002B05D16420043C80
:100C900001F0EAFA142CEFD10020FFF701FD16480D
:100CA00001F000FF192001F0DFFA01F0B7FD002884
:100CB00002D0FFF7C1FB02E0013C002CF2DC02F0A5
:100CC000EFFA03F0B9F91E2300930F2301930B48A9
:100CD0000B490C4A0C4B03F0C1F90C4803F0F0F936
:100CE000FFF792FE74400440984004409C4004404A
:100CF0009440044048010010835300001D50000040
:100D000001030000750600008C020010780200103C
:100D1000F7B500283BD00378303B5A425341C01806
:100D20000378782B03D101301026012501E00A2633
:100D300000250378002201922D2B02D101230130DE
:100D4000019300230278002A1BD0171C303FFCB20D
:100D5000092C02D87343DB1911E020273A43002DF8
:100D600008D0171C613FFFB2052F03D81B01573A6B
:100D7000134304E0064801F095FE002007E001302F
:100D8000E0E7019A002A00D05B420B600120FEBD23
:100D90008D5300000378202B01D10130FAE7704712
:100DA000031C303BDAB2092A01D8181C0AE02023C0
:100DB0001843031C613BDBB2052B01D8573801E017
:100DC00001204042704770B50E1CFFF7E3FF00257D
:100DD000041C2078002807D0FFF7E2FF002803DB7F
:100DE0002D0105430134F4E73560201C70BD00007F
:100DF00008B500F023FD011C014801F053FE08BDB9
:100E00009B53000000B589B0684602F08DF8694632
:100E1000024801F047FE09B000BDC046D7530000AC
:100E2000F7B50F1C01A9161CFFF772FF002814D09C
:100E3000019C0B49201C04F0F1F90D1C081C6421D5
:100E400004F0ECF9281C3970642104F091F904498C
:100E50003070201C04F08CF901E001204042FEBDFE
:100E60001027000037B50D1C48686A4669460731EF
:100E70000632FFF7D5FF01AC69466A462080013291
:100E8000A8680231FFF7CCFF6B4618702288044B2C
:100E90009A4203D9201C694602F0D5F837BDC046F6
:100EA0006B07000007B5486801A9FFF731FF019BF8
:100EB0003C20584302F0E0F807BD000007235843E8
:100EC000054A10189C30013B04D3C25C002AFAD0BA
:100ED000002000E001207047CC04001030B5194814
:100EE00085B001F0DFFD0024651CA30719D1201C8B
:100EF000FFF7E4FF002810D0281CFFF7DFFF0028D1
:100F00000BD0A01CFFF7DAFF002806D0E01CFFF78B
:100F1000D5FF002801D004340EE00B48211C01F05D
:100F2000C1FD211C684602F0CFF9684601F078FE49
:100F3000064801F0B7FD2C1CFF2CD5DD01F07EFE2C
:100F400005B030BDA0520000A7530000999B0000DF
:100F500070B50E1CFFF71EFF0D25041C0134631E27
:100F60001878FFF71DFF002806DB7055013DF5D20C
:100F7000201CFFF70FFF00E0002070BD70B5444C4F
:100F800086B023680868251C002B06D1414801F073
:100F900089FD03F051F8012309E0012B0DD13E49F1
:100FA000082201F0EEFD002803D1236801332360FD
:100FB0006BE03A4801F076FD5FE00378412B17D1F2
:100FC000374C0230211CFFF7C3FF002855D00378AF
:100FD000422B52D1211C02300E31FFF7B9FF0028FD
:100FE0004BD00378432B48D1211C02301C3103E045
:100FF000532B06D12B490230FFF7AAFF002844D11A
:101000003BE04D2B1FD1284C0230211CFFF7A0FFE5
:10101000002832D003784E2B2FD1211C02300E3104
:10102000FFF796FF002828D00378472B25D1023000
:1010300001A9FFF7C8FE019B002B1EDB184A1B48C5
:1010400053651B491DE001A9FFF7BDFE047820236D
:10105000061C9C4311D1301C02A9FFF779FF019BAC
:10106000061CE118FF2902DC02A802F043F9002E59
:1010700003D00134042CEED107E002F0DDFF0B4871
:101080000C4901F00FFD00232B6006B070BDC04677
:101090004C020010B0530000A0520000C6530000E4
:1010A000CC04001012050010F6040010D25300000A
:1010B000FD520000DC53000037B54C682378002B4C
:1010C00025D0201CFFF766FE01A9FFF77CFE019BDF
:1010D000041C002B1BD0D8B2FF2B09DD00F022FA34
:1010E000019B051C1812C0B200F01CFA019003E02D
:1010F00000F018FA002501900198002802D0291C60
:10110000FFF76AF923785A1E9341E418D6E737BDF2
:10111000064A08B5137801214B40137001D00449E9
:1011200000E00449044801F0BDFC08BD8003001044
:1011300080530000E3530000E753000007B5486800
:1011400001A9FFF7E5FD019B002B01DC01230193C1
:10115000019B1E2B01DD1E2301930199034A044BC1
:101160004A4304481A6001F09DFC07BD7017000057
:101170007C030010F653000038B5051C002D09D083
:10118000642402200021013C00F062FE002CF8D112
:10119000013DF3E738BD70B5061C01200821021C93
:1011A00000F080FE072401200821002200F07AFED2
:1011B000321C012522412A400020022100F072FE4B
:1011C000281C08212A1C00F06DFE013CEBD270BDEA
:1011D00010B50021041C0A1C022000F063FE201C34
:1011E000FFF7D9FF10BDF0B5012385B002930023AE
:1011F000061C039372B6002402AB1B5950204042D8
:101200001843C0B2FFF7E4FF0020FFF7E1FF102012
:10121000FFF7DEFFE020FFF7DBFF21276743002514
:10122000F71902200021012200F03CFE785D013513
:10123000FFF7B1FF842DF4D10434082CDCD162B661
:1012400005B0F0BD08B5AC20FFF7C2FFAE20FFF738
:10125000BFFFA520FFF7BCFF08BD38B50122051C64
:101260000C1C00F0CFFD281C211C012200F01AFEEE
:1012700038BD08B5AF20FFF7ABFFA420FFF7A8FFEC
:1012800008BD08B5AE20FFF7A3FF08BD10B5041CCC
:10129000F820FFF79DFF201CFFF79AFF10BD10B547
:1012A000041C8120FFF794FF3F202040FFF790FFB0
:1012B00010BD000008B5074B20201B781843FFF72E
:1012C00087FF0A20FFF758FF034B1878FFF7E7FF67
:1012D00008BDC046000000103C01001008B5842283
:1012E00002480021520001F017FC08BD81030010E4
:1012F00008B50248FFF777FF08BDC046810300101C
:1013000008B501200821FFF7A8FF00200221FFF700
:10131000A4FF02200021FFF7A0FF02200621FFF713
:101320009CFF0320011CFFF798FF0320011C0022F3
:1013300000F0B8FD02200621002200F0B3FD0621D6
:101340000122022000F0AEFDFFF7C8FFFFF7D0FF3B
:10135000A220FFF73DFFA020FFF73AFFC020FFF7D4
:1013600037FF0020FFF792FF0A20FFF705FF40201C
:10137000FFF72EFF2C20FFF72BFF3220FFF7FCFE9C
:101380002E20FFF725FF3220FFF7F6FE2F20FFF774
:101390001FFF0A20FFF7F0FEFFF78CFFFFF769FF42
:1013A00008BD000083280ED80F290CD8CB08842252
:1013B00053430722C0181140034B80220A41111CDD
:1013C0001A5C11431954704781030010F7B55B187C
:1013D000DBB20193019B994215D28425CC086C4362
:1013E00007270F40802504193D41EFB2A618B442EB
:1013F00006DA054D65192B7801343B432B70F6E76F
:101400000131C9B2E6E7F7BD81030010F0B51E1C3B
:1014100087B00592F27804915B68824201D23078FD
:1014200045E0244AB478934205D10322041B544377
:101430000192E4180CE0001B0022824204DA1978C1
:10144000013202315B18F8E71A789C1C5B78019333
:10145000A218002503922F1C019B9F4226DA082226
:101460000023029200937378009A9A421CDA029A3F
:10147000082A06D1039B9C4218D0002225780292AC
:101480000134EB0708D5049A009BB818059AC0B23E
:101490009918C9B2FFF786FF009B029A0133013207
:1014A0006D1000930292DEE70137D5E7019807B08F
:1014B000F0BDC0461A540000F7B5041C0D1C161CE4
:1014C0001F1C01F04CFB20180190019B9C420BD08B
:1014D000832D09D82078291C321C3B1CFFF796FF6E
:1014E00001302D180134F0E7F7BD000010B50021E0
:1014F000012204230A4C0C5D844203D118010243EB
:10150000D0B20BE0013B002B04D10132092A00DDEF
:101510001A1C042301312829ECD1002010BDC0463B
:10152000E05B00000F23020918408000031F00D574
:101530002833511E0020032906D8242B04DC042163
:101540008A1A0249CB18985C7047C046E05B0000DD
:1015500038B5051C0024054B291CE05C044B013404
:10156000C01800F0C5FC0A2CF5D138BD1C5C000089
:1015700000400440F8B50D4F3C68002C15D11020F8
:10158000FFF7E6FF0A4B0022E65C1B195D78301C72
:10159000291C00F037FC0234301C291C012200F009
:1015A00081FC142CEED101233B60F8BD40010010FA
:1015B000085C000070B500240B4B0122E65C1B198F
:1015C0005D78301C291C00F01DFC0234301C291CE5
:1015D000002200F067FC142CEED10020FFF7B8FFCA
:1015E000024B00221A6070BD085C00004001001030
:1015F00038B5051CFFF7BEFF002D09D007210122D9
:10160000022000F0FFFB104B80211A688A431A6009
:1016100000200B2100F01CFC0124002805D0002034
:101620000B2100F015FC44424441002D09D0072154
:101630000022022000F0E6FB034B80211A680A43D7
:101640001A60201C38BDC046FC3F0250F0B587B080
:10165000002602900120039104960596FFF7C8FF2B
:10166000B04202D01823049301260021284C009197
:1016700020786178012200F0C5FB20786178002293
:1016800000F010FC234B9D1D012E24DC6A782F787E
:10169000111C381C019200F0DBFB002808D10099D6
:1016A0001D4AB3008A5C103369465A5001360BE07C
:1016B0002878697800F0CCFB0028F0D0381C01991C
:1016C00000F0C6FB0028EAD0009A144B0132023D1C
:1016D00000929D42D8D127786578381C291C0022B9
:1016E00000F090FB291C381C012200F0DBFB0C49A8
:1016F00002348C42BCD10020864206D0049A029B60
:1017000005991A60039A0120116007B0F0BDC04628
:10171000085C0000D85B0000E05B0000D65B0000C6
:101720001C5C000008B50120021C0B2100F06AFBC4
:1017300001200B21002200F0B5FB03200221012231
:1017400000F060FB03200221002200F0ABFB08BD8B
:10175000234B37B51A6810218A431A60214B802227
:10176000196892010A431A60051C0B21012000220E
:1017700000F048FB01200B21002200F093FB1A4BE4
:101780009F211A68194C8A431A601A6818491A600E
:10179000184B186803F0ECFC8023000218432A1C45
:1017A00020600221032000F07DFB142000F05CFD8E
:1017B0002368FF229343236023680F4A1343236067
:1017C0000E4B1B680193019B002BF9DA22680C4B2E
:1017D00013402360FFF7A6FF01980004800D3EBD73
:1017E00038820440808004409840044000C001409A
:1017F00000093D0090040010800000012CC0014051
:10180000FFFFFFF810B50C4C2068002813DA002009
:101810002060FFF79DFF0A280ADC0120FFF798FFF0
:101820000138C023FF385B00984201D801232360B0
:10183000FFF778FF206810BD0400001008B5FFF71F
:10184000E1FF002801D1002007E00120FFF780FF21
:10185000011EF8D0014803F08BFC08BD50BB1200FC
:1018600008B5FFF7CFFF00280AD0FFF7E7FFFA22FD
:10187000031C0021C00FD2009A424841014B18605E
:1018800008BDC0464401001008B5074B02221A608B
:10189000064BA2221960064B1A70A32258709A7048
:1018A00000F0F2FD08BDC046BC0400109804001012
:1018B000AC04001008B5064B02311960054B00223C
:1018C0001A60054BA2221A70587000F0DDFD08BDA9
:1018D000BC04001098040010AC04001070B5051C86
:1018E0000E1C0324281C311CFFF7CEFF0223FF33FC
:1018F000984202D0013C002CF4D170BD70B5051C9B
:101900000E1C0324281C311CFFF7D4FF0223FF33D5
:10191000984202D0013C002CF4D170BD0B4B10B5A5
:101920001C6800239C420ED0094CA31CA270140A10
:101930005C70140C120EDA709C70FFF7DFFF831ED0
:10194000FF3B5A425341181C10BDC04648010010CD
:10195000AC04001070B50E4C25680024A54215D0CB
:101960000C4C160AA270E670160C120E6271A3716E
:10197000A21D26711C0A54701C0C1B0E9470D3708F
:10198000FFF7BCFF841EFF3C63425C41201C70BD1E
:1019900048010010AC04001008B5064B1A6800237B
:1019A0009A4205D0FFF79AFF831EFF3B5A425341EC
:1019B000181C08BD4801001008B5074B00201B6823
:1019C000834207D002200721FFF788FF0238FF3843
:1019D0004342584108BDC0464801001038B50F4B7E
:1019E000051C1B680020834217D00924641B631E5A
:1019F000062B10D8072C05D00948A91E0918221C4F
:101A000001F068F8E8B2211CFFF778FF0238FF38D0
:101A10004342584101E00120404238BD48010010D6
:101A2000AE040010012010B5011CFFF757FF022380
:101A3000FF3398420ED1094B01211960084B1C78E5
:101A4000230709D0074B032222409A70081CFFF796
:101A500055FF01E001246442201C10BD4801001024
:101A60009C040010AC04001008B5FFF7DBFF022057
:101A70000121FFF733FF0223FF3398420FD1084BB8
:101A80001B787F2B06D98422022007215204054BA4
:101A9000FFF760FF09200421034AFFF73FFF08BD5D
:101AA0009C040010020114008080808010B5002882
:101AB0000CD0254B80211A688A431A60234B1B687F
:101AC000D907FBD5224B03221A6001E0204B186096
:101AD000204B012200211A6019601A601968012246
:101AE0001142FBD01C4B80211A601C4A4902146829
:101AF000214311601A1C002804D1134B802419685B
:101B000021431960164B196888421CD018600028C0
:101B100001D0144800E01448116803F0DBFA134BBD
:101B2000FA2118608900041C03F022FB1E2358438D
:101B30000F4BC82118604901201C03F019FB0D4B05
:101B4000186001F03DF810BD388204400C8004405C
:101B50007080044074800440788004408080044099
:101B600008000010006CDC02001BB700900400109D
:101B70008C0400109404001008B500F035F9134BE4
:101B800000211A68120B12031A60114B1A68120B0B
:101B900012031A600F4B1A68120B12031A600E4BD5
:101BA0001A68120B12031A600C4B012219600C4BBD
:101BB0001A6019601A601A6801200242FBD0094BB2
:101BC00023221A60FFF772FF08BDC0460080005054
:101BD000008001500080025000800350408004408B
:101BE000448004400880044038B50F490F4800F095
:101BF00059FF0F4D0024281C00F054FF0D4A0E48D9
:101C0000A1581219D2682B1C143400F04BFFC82CB9
:101C1000F4D10A4800F046FF00F046FB011C0848DA
:101C200000F040FF38BDC046A0520000265C000016
:101C3000765C00006C5D0000385C0000435C0000D6
:101C4000655C0000F0B53B4B8BB01E68041C002E99
:101C500001D1351C08E0384B02901B6801209B68BD
:101C600054E033681E79019D2378002B31D0082D74
:101C700033D02378202B01D10134FAE7002B28D070
:101C80006A1CAD0008356B460192EC50FF2E4CD01B
:101C90002278002A07D0631C202A01D01C1CF7E7F9
:101CA000002222701C1C019A012ADCD1224E234BF7
:101CB0000B253360371C013D002D2ED03B68029868
:101CC000196800F06FFF0028CBD03B6814333B60ED
:101CD000F1E7002D1CD0022D02D0B54206D911E04B
:101CE0000398174900F05EFF0028F6D1124C154802
:101CF0002368D96800F0D6FE23681348196900F0FC
:101D0000D1FE05E00C4BE8B21B689B6802A998471E
:101D1000084A1368002B0BD103E0281C291CFFF78D
:101D200063FF0A4800F0BEFE02E0019D0026D2E7F4
:101D30000BB0F0BD4C020010540200106C5D0000AE
:101D4000CD520000725C0000D7530000795C0000A7
:101D500038B5041C164D0A2808D002D8082811D01E
:101D60001CE00D2802D07F280CD017E02A68002341
:101D70001370104800F096FE0F4C201CFFF762FF16
:101D80002C6013E00C4B2A689A420FD90B48211C97
:101D900000F088FE2B68013B2B6007E00748211C00
:101DA00000F080FE2B685A1C2A601C7038BDC046AB
:101DB00050020010765C00004C010010855C0000B1
:101DC00008B500F02BFD002804D000F0FDFCFFF763
:101DD000BFFFF6E708BD0000014A024B1A607047DA
:101DE0004C01001050020010044B40211A680A43B5
:101DF0001A60034B01221A707047C046808004406D
:101E0000580200100F4B70B51B78061C0C1C151CDB
:101E1000002B01D1FFF7E8FF701E022803D80A4B00
:101E20008000C35800E0094B1A68012D04D1A54079
:101E30002C1C14431C6003E00121A1408A431A605A
:101E400070BDC04658020010345E00000080005093
:101E500038B50F4B051C1B780C1C002B01D1FFF76C
:101E6000C3FF0020032D12D8281C012203F01EF905
:101E700002040608074B04E0074B02E0074B00E0B2
:101E8000074B1B68A2401340181C421E904138BDEE
:101E900058020010FC3F0050FC3F0150FC3F025034
:101EA000FC3F03500F4B70B51B78061C0C1C151C17
:101EB000002B01D1FFF798FF701E022803D80A4BB0
:101EC0008000C35800E0094B1A68012D04D1A540D9
:101ED0002C1C14431C6003E00121A1408A431A60BA
:101EE00070BDC04658020010405E0000FC3F00502C
:101EF00038B5084B041C1B780D1C002B01D1FFF7D3
:101F000073FF236818229343236023681D432560D1
:101F100038BDC04658020010054B3F221A60054BE1
:101F200001221A60044B40211A688A431A607047E4
:101F300024800440D88004403882044008B5044B13
:101F400040211A688A431A60FFF7E6FF08BDC046C1
:101F50003882044008B500F05DFAFFF72BFB0A4811
:101F60000021FFF7C5FF09480021FFF7C1FF08481E
:101F70000021FFF7BDFF07480021FFF7B9FF064822
:101F80000021FFF7B5FF08BD0840044000400440B1
:101F9000AC400440144004401C40044008B50120FB
:101FA000FEF750F908BD000008B5124B8022DA6731
:101FB0005200DA678022D200DA6780225201DA67A3
:101FC00080221201DA6780229200DA670A4A00232F
:101FD00013600121094A49421160094A1360094A04
:101FE0001360094A01231360084A1360FFF7D6FF04
:101FF00008BDC04604E100E00482044008820440B9
:1020000004C000403CC0004000C00040004001400F
:1020100008B5064B1A6801321A60054B1868FFF7BD
:1020200045FDFFF7C1FFC046C04608BD5C02001079
:1020300008000010F7B5071C0C1C72B6FFF78AFFEA
:10204000524B1A68524B1A60002F01D0514B00E0DE
:10205000514B524A04211360514B524D1A680A43A6
:102060001A6000232B60A1071ED04F4B4F4A1968FE
:102070000A401A6029684E4BA2070ED5EC22520185
:102080000A432A6080221A6052001A608022D2001D
:102090001A60802252011A6003E0802212010A4372
:1020A0002A60802212011A60002F53D0414B002475
:1020B0001C60414B414E1C60414B301C1C60414B2D
:1020C000211C1C60FFF714FF201C0921221CFFF7B4
:1020D00099FE201C0921221CFFF7E4FE3A4B8021C7
:1020E0001A683A480A431A603368072293433360F8
:1020F00033680222134333600A21784302F0EAFF77
:10210000334B03221860334B1C60334B1A60334B44
:10211000334A19680A401A601A6880210A431A6013
:10212000234A8B001360204A1168194311602A6802
:10213000022113432B602B4B01221A602A4B19609A
:102140002A4B1C491A601C601A6018680122104250
:10215000FBD00A60264B012252421A60254B002216
:102160001B680193244B1A6062B630BFC046214BF6
:10217000019A1B689A4208D11F4B01221A601F4B1B
:102180001868FFF793FCFFF70FFFF7BD3882044094
:1021900034820440BF180000FF1800003082044061
:1021A00010ED00E004820440008204407FE2FFFF63
:1021B00000E100E004C0004004000140644004402D
:1021C000044001400480014080800440841E0000DF
:1021D00018C0004008C0004014C000403CC000408F
:1021E0000FF0FFFF7880044070800440748004404A
:1021F000088204405C020010600200100800001019
:1022000008B5FFF717FF08BD074B1A68013203D165
:10221000064A1168013111601A6801321A60044BD4
:102220001A6801321A607047700200106C020010C8
:1022300064020010074B98420AD8074A0023136033
:10224000064A01381060064A1360064B07221A60DE
:102250007047C046FFFFFF007002001014E000E06E
:1022600018E000E010E000E00B4A10B51368002809
:1022700000D10120C1438B4208D91168994209D38A
:10228000591C146809188C42FAD3F6E71168C91A68
:102290008142FBD310BDC04670020010014B18688C
:1022A0007047C04670020010064BFA211868064BB2
:1022B00010B589001C6802F00DFF044B5C43201828
:1022C00010BDC046700200106C020010378941003A
:1022D000034B01221A60034B1A6801321A607047DF
:1022E00000C0004074020010034B01221A60034B2F
:1022F0001A6801321A60704700000140780200102D
:10230000002803D1044B01221A6003E0012801D107
:10231000024B18607047C04604C0004004000140F2
:10232000002802D1044B186004E0012802D1034BBD
:1023300000221A607047C04604C0004004000140FB
:10234000002801D1044B02E0012804D1034B1A6894
:1023500002210A431A60704704C000400400014093
:1023600010B5002900D1134900280DD1124B80244B
:102370001A6822431A60114B03221860104B19602F
:10238000104B1A60620211E0012811D10A4B802221
:102390001868520002431A600B4B00221A600B4B64
:1023A000032219600A4B1A6080229202094B1A60BC
:1023B00010BDC046FFFF0000808004407402001082
:1023C00018C0004014C000407802001018000140FE
:1023D0001400014000E100E080231022DB051A60B8
:1023E000094B08221A6000238022D2051268D10608
:1023F00004D5064A934201D00133F5E704489842D8
:102400009B4158427047C04618000040FF0F000033
:10241000FE0F000008B58022154B1202DA67154B3B
:102420006C221A60144B154A19680020114019607B
:1024300019681960124B19680A401A601A68042159
:102440001A600122FFF7DEFC002004210122FFF7C1
:1024500029FD002005210122FFF7D4FC01220020E4
:102460000521FFF71FFD074B00221A6008BDC0467B
:1024700004E100E01800004030400440F8FCFFFF99
:102480003440044004800440F8B5174A174C002338
:1024900023601360164A202113608022D205116048
:1024A0002168144A012903D0934203D00133F7E78E
:1024B000934203D1FFF790FF002014E00E4F002558
:1024C0003E68013E2368FF2B0CD83B689E4204D037
:1024D0003E68FFF7E3FE051C0A35FFF7DFFE854285
:1024E000F0D1E7E72068F8BD7C0200108002001000
:1024F00084020010FF0F000088020010034B01222D
:102500001A60034B1A6801321A607047004001409C
:102510008C020010174B70B501241C60164B1A6812
:1025200012191A60154B1A68002A22D01A68144D25
:10253000013A1A601E68002E0DD02A68201C211C4A
:10254000FFF7B0FC2B68201CE31A2B602A680221DD
:10255000FFF7A8FC0DE01B68201C2B602A68211CDB
:10256000FFF7A0FC2A68201C0221FFF79BFC054B0B
:102570001E6070BD008001409402001090020010A7
:102580009802001004800140002803D1044B01226E
:102590001A6003E0012801D1024B18607047C04661
:1025A0000440014004800140002802D1044B18601F
:1025B00004E0012802D1034B00221A607047C04694
:1025C0000440014004800140002801D1044B02E096
:1025D000012804D1034B1A6802210A431A6070478C
:1025E000044001400480014010B500280FD1124B77
:1025F00080221C68920022431A60104B032218604C
:102600000F4B19600F4B1A608022D20211E0012893
:1026100011D1094B80221868D20002431A600A4B7C
:1026200000221A60094B03221960094B1A608022AC
:102630001203084B1A6010BD808004408C02001009
:1026400018400140144001409402001018800140DD
:102650001480014000E100E008B5184B1A680E2311
:102660001340062B0DD1164B9E221B68134205D03A
:10267000144ADBB25360144B1B681EE0D9071CD50B
:1026800001E0042B05D1104B1868C0B200F0B1F87E
:1026900013E00C2B06D10B4B8022596852000A43E1
:1026A0005A600AE0022B08D1054B1A68054B9106C7
:1026B00001D5002200E001229A6008BD0880004098
:1026C000148000409C0200100080004000487047C9
:1026D0009C020010F7B52D4B2D4C80220021920357
:1026E0000191061CDA67201C902200F015FA019B6C
:1026F0000725A360274B284F1A68AA431A60196858
:10270000012211431960254B1968A9431960196802
:1027100011431960224B8021186849010143196057
:10272000204B1A6083223A601F4A126819681F4BB7
:102730001868504302F0CEFC311C000902F0CAFCBC
:102740001B4B10221B491A60030A0B601A4BC0B2C4
:10275000032218603A60194A1560194A1D1C106856
:102760000190106860230340602BFAD110680123A8
:10277000184202D02B680193F8E723708022114B96
:1027800092031A6005230B60F7BDC04604E100E028
:102790009C020010A44004400C800040A84004406B
:1027A00080800440988004407880044090040010A9
:1027B00028800040048000400080004008800040E5
:1027C0001480004000E100E008B5FFF77FFFC26819
:1027D000031C1202120E8218D07BDA681202120E4B
:1027E0000132D2B29A7352B2002A01DA00229A73ED
:1027F00008BD10B5041CFFF769FFC2681204120E71
:102800008218D473C2681204120E0132D2B242731B
:1028100052B2002A01DA0022427310BD08B5FFF758
:1028200055FFC268C36812021B041B0E120ED01A99
:10283000431E9841C0B208BD70B500241D5D061945
:10284000002D02D005550134F8E7121B301C131C73
:10285000002B03DD0170013B0130F9E7D043C017C5
:102860000240A01870BDF7B5051C01910093561EDB
:10287000092B01D8041C0CE000980A2102F02AFC64
:102880000199031C321C281CFFF7EDFF071C2C18B4
:1028900007E0671B002E04DD019B013E237001341D
:1028A000F7E700980A2102F059FC3031781C2170BA
:1028B000FEBDF8B50C1CD9175F18051C4F40561EFD
:1028C000092F12D9381C0A21002B03DA02F002FC6E
:1028D000434202E002F0FEFB031C281C211C321CB8
:1028E000FFF7E7FF041C2D1814E0002B00DA961EFA
:1028F0002A1CA919891A002902DD14700132F8E78F
:10290000F443E41734402D19002B03DA2D232B70E8
:1029100001340135381C0A2102F020FC30312970C5
:10292000601CF8BDF7B5089F1E1C051C013A3B0949
:1029300001D1041C05E00093331CFFF7F3FF2C18B2
:1029400006E0601B002A03DD2170013A0134F8E73C
:102950000F231F40092F01D8303704E0002E01D08B
:10296000373700E0573727700130FEBDF0B585B02E
:10297000041C029101D0002101700025117800296A
:1029800006D1029F0023BD426CD22370281C6FE049
:10299000029FBD42F5D2252902D00132217004E008
:1029A0005178252904D12170023201350134E5E73F
:1029B000302902D0561C202100E0961C32782D3A96
:1029C00050424241B6180022307830277F423F18EB
:1029D000FFB2092F07D80A277A438218D2B2303AB9
:1029E000D2B20136F0E7AF18BC46029FBC4501D910
:1029F0007A1BD2B2692818D00BD863282AD0642851
:102A000013D0582832D11F1D1B68201C00930123AE
:102A10001DE075280FD0782814D0732826D11F1DEB
:102A2000201C1B68FFF708FF0AE01F1D201C1B6805
:102A3000FFF73FFF04E01F1D201C1B68FFF713FF7B
:102A40003B1C0BE01F1D1B68201C00930023FFF79D
:102A500069FFF5E71868043320700120721C241800
:102A60002D188BE7013C2370681E01E001204042D5
:102A700005B0F0BD10B50C1C131C6421221CFFF71F
:102A800075FF10BD00B5031C9BB00A1C01A8191CE2
:102A9000FFF7F0FF632800DDFEE701A800F0B6F8BD
:102AA0001BB000BD0FB407B504A908C9181C0191DB
:102AB000FFF7E8FF03B008BC04B018470EB403B535
:102AC00003AA08CA191C0192FFF7D4FF02B008BC80
:102AD00003B0184730B50C1C044303232340041CE7
:102AE000002B01D0002310E0032AFBD9CC58C4509E
:102AF0000433D41A032CF9D8131F9B0801339B000D
:102B0000C418C91803231A40ECE7934203D0CD5CE4
:102B1000E5540133F9E730BD30B5031C840701D11A
:102B2000032A01D89A1814E00B060C041D1C254337
:102B30000D430C022543031C20C38418E41A032C04
:102B4000FAD8131F9B0801339B000324C3182240AB
:102B5000E8E7934202D019700133FAE730BD021C56
:102B6000031C981A0133591E09780029F9D17047BE
:102B7000031C0A781A70002A02D001310133F8E7E9
:102B8000704730B50023934208D0C45CCD5C651B10
:102B900006D10133002CF6D1201C02E0002000E019
:102BA000281C30BD10B50022835C8C5CA34204D18C
:102BB0000132002BF8D1181C00E0181B10BD0000DA
:102BC00008B5094BFA211868890002F0D1FAFFF71D
:102BD00031FB96200002FFF77DFD0120FDF732FB5F
:102BE000FEF742FF08BDC0469004001008B5FEF78E
:102BF000C3FFFFF7F9F8FFF7A1F9FEF781FBFEF736
:102C00006DFBFFF7DDFFFFF7E7F808BD10B5041C0B
:102C10002078002803D00134FDF764FBF8E710BDED
:102C200038B5051C0E24013C04D3295D0248FFF78A
:102C300039FFF8E738BDC0464C5E000038B519488A
:102C4000FFF730FF184C201CFFF7EAFF174D422119
:102C5000281CFFF727FF201C0E30FFF7E1FF432160
:102C6000281CFFF71FFF201C1C30FFF7D9FF10485E
:102C7000FFF718FF201C4630FFF7D2FF0D48FFF783
:102C800011FF201C2A30FFF7CBFF281C4E21FFF735
:102C900009FF201C3830FFF7C3FF616D0648FFF7BE
:102CA00001FF38BD4F5E0000CC040010555E0000EF
:102CB0005C5E0000625E0000685E000003110A2294
:102CC00053430F2210401818704738B50A21041CCE
:102CD00002F04EFA0A210501201C02F09FFA281C7E
:102CE000084338BD08B5C12252000E200221FEF76C
:102CF00015FE024B01225A7108BDC046C0040010E7
:102D000010B5084C6379002B01D1FFF7EBFF237955
:102D10000C221A43A37901205B001A43011CFEF721
:102D2000FDFD10BDC004001010B5074C2379002B29
:102D300008D16379002B01D1FFF7D4FF0123237160
:102D4000FFF7DEFF10BDC046C004001008B5054BFC
:102D50001A79002A05D000221A711A72DA70FFF768
:102D6000CFFF08BDC004001010B501210220FEF7FE
:102D700013FE064B041C18787F231840FFF79EFFB4
:102D8000034B5870DC71201C10BDC0469C04001021
:102D9000C0040010014B01229A707047C00400105B
:102DA000024B00229A701A727047C046C00400108D
:102DB00008B5FFF7D9FF094B094A9978002908D0CF
:102DC000197A012901D8013103E01068054908602A
:102DD00000E019720021D970116008BDC004001014
:102DE000640200106802001008B5FEF71BFE0C23F9
:102DF000184003D0024B1A781043187008BDC04623
:102E0000C004001010B5FFF7EFFF054B1A781C1C2B
:102E1000530701D5FFF7CCFF0023237010BDC04638
:102E2000C004001008B50020FEF7E2FB002801D026
:102E3000FFF7E8FF08BD000010B5054C0023E37163
:102E4000FFF7F0FFE379002B01D1FFF78DFF10BDF5
:102E5000C004001008B50948092102F0EBF9084B3D
:102E6000FA22D2001A80FFF7E7FF064B00221A6011
:102E7000FA22054B92001A6008BDC046C00400103B
:102E8000CA040010640200106802001008B5FFF7C1
:102E9000C9FF002008BD08B5FFF758FF08BD0000B6
:102EA00070B51D4C061C637822781B021343A27870
:102EB000A07912041343E2780D1C12061343174A3B
:102EC00013401A0A237062701A0C1B0EE3706379A8
:102ED000A27022791B021343114A134023711B0A6B
:102EE0006371FFF7EBFE0F4B1B88C01830806079D1
:102EF000FFF7E4FEB070E078FFF7E0FEF070A07836
:102F0000FFF7DCFE28706078FFF7D8FE6870207845
:102F1000FFF7D4FEA87070BD9C0400107F7F3F3F78
:102F2000071F0000CA040010F0B58DB0051CFEF7A5
:102F300043FD002804D1281C1249FFF7BFFD1EE005
:102F40000AAE0BAC211C301CFFF7AAFF3388F778C0
:102F50000793B378267808936378A47809930A4B8B
:102F6000187900F0D7F8099B049002930097019616
:102F70000394281C0549079A089BFFF79FFD0DB095
:102F8000F0BDC046745E00009C040010795E000035
:102F900070B5061C0D1C141CFEF70EFD00280AD08F
:102FA000301C291CFFF77CFF002C07D0044B0020AD
:102FB0001B79236003E00120404200E0201C70BD2B
:102FC0009C040010F7B504880E1C051C6421201C0D
:102FD0000092019302F0C2F8114B8FB2B078E41B5B
:102FE0001C80FFF772FE0F4CA0707078FFF76DFE2B
:102FF000E0703078FFF769FE2071E878FFF765FE32
:10300000009B6071A371A878FFF75FFEE071381C28
:10301000FFF75BFE20720198FEF7E0FCFEBDC046A4
:10302000CA040010AC04001008B50223FFF7CAFF61
:1030300008BD08B5021C501E82415201002001212A
:10304000FEF76CFC08BD38B5041C01200D1CFFF711
:10305000F0FF201C00F086F8072102F0DFF8201CAA
:103060000A1C291CFFF7E0FF96204000FFF7FCF840
:103070000020FFF7DEFF38BD73B5041CFFF774FEB8
:10308000002801D100203BE01E4B5D781E1C7378A8
:10309000AB4207D10A20FFF7E7F8FFF765FE0028EB
:1030A000F5D1EFE7FEF788FC0028EBD001A96846D0
:1030B000FFF7F6FE684600F055F8051C01A800F081
:1030C00031F8114B04199C420DD9E3170122134327
:1030D000ED18281C694600F075F8002C01DA0B4B3E
:1030E00000E00B4BE418201C01A900F024F8281C78
:1030F000072102F093F868460A1C01A9FFF794FF24
:1031000076BDC046C00400107F510100805101000F
:1031100080AEFEFF07231840014B8000C058704767
:10312000EC5E000002783C235A4341785218534326
:1031300082789818704738B50C1C3C21051C02F0A9
:103140006DF8281CA1703C2102F012F83C2102F01D
:1031500065F86170E121281C090102F009F820706E
:1031600038BD000070B58378022100229942524197
:10317000048896214901051C64180C20A41A4243B6
:103180009B18033B992058430521023001F0F0FFC2
:103190006E26FF3666436421A31086194942201C1F
:1031A000F61801F0E5FFC82136184900201C01F08F
:1031B000DFFF034B3018C018EB78C01870BDC04655
:1031C000D382FFFFF8B5204B0C1CC5181F4B8000A5
:1031D000C0181F4901F0CCFF03235843C617B60F90
:1031E0003618B610AE19B600953E301C194902F0DB
:1031F00015F8CD17AD0F6D180527AD107D430235BD
:10320000281C992102F00AF8081C391C01F0B0FFB3
:103210000130E0709921281C01F0AAFF0C21023036
:1032200001F0FCFF4D1CEDB2A570301C094901F006
:103230009FFF094B0C21C6180E20401B01F098FF80
:1032400036182680F8BDC04679050000652F0400B9
:10325000B13A0200B505000094EDFFFFF8238A01A2
:10326000DB0013404A05920E1343F822120211406C
:1032700019430A23594330B5CA1083181C1CEB3478
:103280005D782478EA336C401B7824021C43835C0D
:10329000201C58400723194008418005800D30BD8F
:1032A0007047000008B5054B011E994201DD044B33
:1032B000C1180448EA38FFF7D1FF08BDFF17000026
:1032C00000F8FFFF285F00000723594310B5084BA3
:1032D00059189C310023CC5C0F2222400270CA5C3A
:1032E0000133120942700230072BF4D110BDC046E1
:1032F000CC0400100723594310B5074B59189C31D3
:1033000000234278047812012243CA540133023068
:10331000072BF6D110BDC046CC04001070B5AD4CE3
:1033200086B0E36E6E465A1E934117363370AA4B31
:103330009A6A191CD006400F0138062807D801F0F8
:10334000B5FE040C2012181A1D00022509E0636E58
:1033500016339B001B591D1C15E0636E16339B0032
:10336000E55800230FE0A36DE56DAB420BDD0D25A5
:1033700009E0022503E00C25032304E00D252B1CA6
:1033800001E00D25EDE70D6150111F2800D91BE16B
:1033900001F096FE2000220029002C002F003300AF
:1033A0003B00440048004C00540061006E00760071
:1033B00083008F009B00A800B800C500D500D30093
:1033C000E100E400E700EF00FE0002010B010D0147
:1033D0000F011501E01801E0E0180E30EB1A591C3E
:1033E00001F028FFF0E0E0181C30F7E7211C0E3157
:1033F00005E0E0180E30E1180BE0211C1C31201C08
:103400001A1C2B1C01F095F9DEE0E018E1181C30C5
:103410000E31EB1A5A1CFFF75DFBD5E06F48011C1B
:103420000E31EDE7E018011C1C31F2E7226E10218D
:10343000002A00D00A21221C0E3206E0226E102142
:10344000002A00D00A21221C1C320291009501960C
:10345000201C211C53E0216E012232701022002911
:1034600000D00A22009501960292201C211C45E002
:10347000226E1021002A00D00A21221C0E3213E0F5
:10348000216E012232701022002900D00A220095FC
:1034900001960292201C211C4DE0226E1021002A70
:1034A00000D00A21221C1C32009501960291201C9A
:1034B0006AE0226E1021002A00D00A21484A0291B7
:1034C00000950196101C111C19E0216E1020002996
:1034D00000D00A20424A0290111C1C390095019626
:1034E000101C0CE0216E012232701022002900D045
:1034F0000A223B49009501960292081C002201F025
:1035000022F961E0226E1020002A00D00A20344AFD
:103510000290111C1C3900950196101C35E0216E9B
:10352000012232701022002900D00A222C49009575
:1035300001960292081C002227E001223270226EBE
:103540001021002A00D00A21254A029100950196F7
:10355000101C002119E0009620481BE0009620482E
:1035600018E0226E1021002A00D00A21221C1C32F1
:1035700006E0226E1021002A00D00A21221C0E3201
:103580000095019602910020211C01F004F91BE036
:103590000096201C002103E0211C1C310096201CF9
:1035A0001A1C2B1C01F05AF90EE0201C02E00B48FB
:1035B00000E00B48191C2A1C01F067F904E0201CEC
:1035C000191C2A1C01F06BF933780120E36606B060
:1035D00070BDC046CC040010680C0010DA04001066
:1035E000E8040010064910B50A1C883213681C1C38
:1035F0001E34A4006050013303210B40136010BD42
:10360000CC040010054B0322191C883108680138CE
:1036100002400A601E329200D0587047CC0400105D
:10362000F7B5124F3D1C8C3528680130FFF73AFE84
:103630000F4EBB6EB26A041C01920122F06202407E
:103640009A4210D1830703D428680230FFF7CAFFDB
:10365000FF239B00019A1C40A40193101C438C374C
:1036600001233C60F3600220FEBDC046CC04001084
:10367000680C00100C490D488A6A031C8C3370B525
:103680001D68D3059B0E0C1C910500D5403B866E32
:10369000921001210A40B24203D18C30EB18036032
:1036A000E160012070BDC046680C0010CC04001021
:1036B00008B5084B5A1CD07F9A1CD27F0001120219
:1036C000104303331A7FDB7F10431B031843FFF7BC
:1036D00089FF08BDCC04001008B5FFF793FF032352
:1036E000044A0F219A180140013311770011072B6A
:1036F000F6D108BDCC04001008B5FFF783FF034BDB
:1037000001228C331860024BDA6008BDCC04001033
:10371000680C001010B5064CA36E002B06D0FFF706
:1037200071FF044B8C3401222060DA6010BDC0466A
:10373000CC040010680C001010B5064CA36E002BD2
:1037400006D1FFF75FFF044B8C3401222060DA6062
:1037500010BDC046CC040010680C001008B5044B26
:1037600001221A62034B1B68002B00D0984708BD4A
:10377000680C00102C03001008B5104B0022596A89
:103780001A62914214D05969914216DD012906D17D
:10379000D969914203D0DA610A2299615A615A6962
:1037A000032A02DD06490120C866013A5A6104E095
:1037B000044B1B68002B00D0984708BD680C001014
:1037C000CC0400102C030010074B5A6A002A02D0C8
:1037D0005A69002A07DD9A690F21044B1140D977F5
:1037E00012110133DA777047680C0010CC04001016
:1037F000044B597F9A7F090112020A43197F0A4339
:103800005A677047CC0400100B1C093B10B5012B04
:103810000FD80023074A9A18147FC25C944205D03F
:10382000054B08395A681143596002E001330E2BE9
:10383000F0D110BDCC040010680C001008B50829A8
:103840000DD0192913D1427808231A4202D0002240
:10385000027002E00F2303700723437005E000238A
:103860000022C25401330E2BFAD1FFF743FD08BDED
:1038700030B5114D85B06C6F002802D00F239C43EA
:1038800004436C67FF2C05DD281C1C300E2101F061
:10389000D1FC0FE06846211CFFF716FD6846211C8D
:1038A000FFF7CCFF00236846C15CEA1801331177AB
:1038B0000E2BF8D105B030BDCC040010134B30B541
:1038C000596F0F229143041C0C4385B05C671D1C8B
:1038D000082C19D0FF2C17DC6846211CFFF7F4FCDC
:1038E0006846211CFFF790FF0023EA18127F694603
:1038F000CA5401330E2BF8D16846211CFFF79EFFF6
:103900006846211CFFF7F6FC05B030BDCC04001062
:103910001FB50F4C616F082918D0FF2916DC6846C7
:10392000FFF7D2FC6846616FFFF76EFF0023E218D5
:10393000127F6946CA5401330E2BF8D16846616F75
:10394000FFF77CFF616F6846FFF7D4FC1FBDC046E0
:10395000CC04001010B50D4C631CD87FA31CDB7F7A
:1039600000011B021843E37F1843E31CDB7F1B03AA
:103970001843FFF797FC0F23021C1A40227702110D
:10398000134000126377A07710BDC046CC0400102E
:10399000044B5A6E16329200D258121A51424A41C2
:1039A000DA667047CC040010044B5A6E163292004F
:1039B000D158013900D50D21D1507047CC040010E9
:1039C000054B5A6E16329200D15801310E2900D1A2
:1039D0000021D1507047C046CC040010094B5A6EEC
:1039E00016329200D2580D2A03D11A1C29321278AD
:1039F00005E09A18507F117F0001021C0A435A65A6
:103A00007047C046CC040010084B10B55A6E0F2406
:103A100016329200D1585A6D58181440013104776B
:103A20000D2902DC5B1812111A7710BDCC040010AE
:103A30000E4B30B55A6E596D16329200D2580D2A7F
:103A400007D11C1C2934F0202478084020435865F5
:103A500007E09818447F057F24012C435C650C1116
:103A600044779B180F221140197730BDCC04001009
:103A700008B503480E22011C1C39FFF72BF808BDBE
:103A80000405001008B503480E22011C1C31FFF785
:103A900021F808BDE804001008B504480022011C04
:103AA0001C310D2300F045FE08BDC046E80400109F
:103AB00008B503480E22011C0E39FFF70BF808BDAC
:103AC000F604001008B503480E22011C0E31FFF762
:103AD00001F808BDE804001008B504480022011CE4
:103AE0000E310D2300F025FE08BDC046E80400108D
:103AF0000023044A00219A18463201331170082B22
:103B0000F7D17047CC040010C31C421E0020934222
:103B100007D004494000591846310978013B084351
:103B2000F5E77047CC04001010B50B1D994208D082
:103B3000044A01248A1804404632147040100131AE
:103B4000F4E710BDCC04001038B50020FFF7DCFF0F
:103B5000084C051C0021207FFFF7E6FF0420257795
:103B6000FFF7D2FF0421051C607FFFF7DDFF6577BB
:103B700038BDC046CC04001010B50020FFF7C4FFCC
:103B8000034C20770420FFF7BFFF607710BDC046CD
:103B9000CC04001010B5054C0021207FFFF7C4FFB6
:103BA000607F0421FFF7C0FF10BDC046CC040010A9
:103BB00010B5094C231C8C3318680130FFF772FBD9
:103BC000064B021CD8620F231A40227702111340C1
:103BD00000126377A07710BDCC040010680C0010B1
:103BE00010B5084C0E21201C01F024FB201C0E30C7
:103BF0000E2101F01FFB201C1C300E2101F01AFBCE
:103C000010BDC046CC04001010B50C4B191C0E3171
:103C10001A1C187F1C7801332043D8768B42F8D1C8
:103C2000936E002B08D0064B1B690D2B04D1137F1C
:103C3000111C29310B70537310BDC046CC04001009
:103C4000680C001010B50C4B191C0E311A1C1C7F8F
:103C5000187801332040D8768B42F8D1936E002B30
:103C600008D0064B1B690D2B04D1137F111C293181
:103C70000B70537310BDC046CC040010680C0010CC
:103C800030B5002185B00E4B421C1818007F6C46E1
:103C900008550D25D40F181C002395425C41644241
:103CA000013122400E2901D0101CECE76C46E15C8A
:103CB000C218013311770E2BF8D105B030BDC046C4
:103CC000CC040010074B10B55A6E16329200D4582F
:103CD000611E1C19D1502077002901DA0D21D15025
:103CE00010BDC046CC040010034A0023111C9431BF
:103CF00098320B6013607047CC040010034B012214
:103D0000943319684A401A607047C046CC040010CA
:103D1000044A002313678C321360034B0122DA60DC
:103D20007047C046CC040010680C001008B59E4BCC
:103D30000F20996A9D4A8B101840891101385256FC
:103D40000E2848D801F0B2F9080F171F234729475A
:103D50004731474747353900002A3CDB944B9A18D6
:103D60004032002305E0002A35DB914B9A1840329F
:103D7000012393712DE0002A2DDB8D4B9A184032E0
:103D80009279DA6625E0081CFFF79CFF21E0002A03
:103D900021DB101CFFF7FCFD1BE0002A1BDB844B22
:103DA000596E16318900CA5013E0081CFFF786FDD2
:103DB0000FE0081CFFF75CFD0BE0002A0BDB101C7A
:103DC000FFF75EFF05E00C2B23DD162B28D1FFF754
:103DD00005FE0120EEE0982B03D1754B00221A66F8
:103DE000F7E7982B6CDC382B03D1714B0120586618
:103DF000E0E0382B30DC1C2B02D1FFF739FEE8E77E
:103E00001C2B12DC0C2BDED1694B0120983318607F
:103E1000D0E00120002B00D1CCE001204042C9E0DD
:103E2000182BFAD1FFF774FFD3E7282B03D1604B8F
:103E300000225A66CDE7282B04DC262BEDD1FFF7B4
:103E4000E3FDC6E72C2B02D1FFF71CFEC1E7362BA2
:103E5000E3D1FFF7EDFDBCE7662B02D1FFF732FEA1
:103E6000B7E7662B16DC4C2B03D1FFF7A1FE02202F
:103E7000A0E04C2B04DC3C2BCFD1FFF70DFEA8E7D4
:103E8000562B02D1FFF714FEA3E75C2BC5D1FFF739
:103E90000FFC9EE76C2B02D1FFF71EFC99E76C2B01
:103EA00004DC682BB9D1FFF79BFE92E7762B02D199
:103EB000FFF712FE8DE7882BAFD1FFF785FC88E76F
:103EC000E62B02D1FFF758FE83E7E62B35DCC82B43
:103ED00002D1FFF713FF7CE7C82B16DCA82B03D118
:103EE000334B0120186665E0A82B04DC9C2B94D191
:103EF000FFF77EFC6DE7B82B02D1FFF7F5FE68E710
:103F0000BC2B8AD1FFF704FD63E7D62B02D1FFF764
:103F100041FE5EE7D62B05DCCC2B00D07DE7FFF71A
:103F200019FD56E7D82B02D1FFF7F4FB51E7DC2B44
:103F300000D072E7FFF768FE4BE7F32B02D1FFF7E3
:103F40001BFC46E7F32B17DCEC2B02D1FFF77AFEC4
:103F50003FE7EC2B05DCE82B00D05EE7FFF7ECFB3E
:103F600037E7F12B02D1FFF7C3FD32E7F22B00D088
:103F700053E7FFF7F3FB2CE7F62B02D1FFF7E4FD45
:103F800027E7F62B05DCF52B00D046E7FFF70CFD05
:103F90001FE7F72B02D1FFF713FD1AE7F82B00D02C
:103FA0003BE7FFF7A9FB14E7680C0010289B000013
:103FB000CC04001008BDC04638B5184C231C8C3307
:103FC0001868FFF76FF9164B0022E16EDA60E266BF
:103FD00003229862A16610401D1C022809D090425D
:103FE0000AD0012802D0FFF7A1FE07E0FFF718FB77
:103FF00004E0FFF793F901E0FFF73CFB00280BDD3D
:10400000EB68002B04D1231C8C3319680A181A6042
:10401000903422681318236038BDC046CC040010C9
:10402000680C0010034B0122DA660F229A775A7748
:104030001A777047CC04001010B5054C0549201CB8
:1040400001F0F8F8FFF7EEFF0123636610BDC046EC
:10405000CC0400109C0700007047000030B50C4DE8
:10406000049C28600B4801600B490A600B4A1360EE
:104070000B4B039A1A600B4B0B4A1C600B4B1C60DA
:104080000B4B1A600B4B0C4A13600C4A136030BD8B
:104090005803001068030010740300103C03001064
:1040A0003403001010000010CD410000680C001017
:1040B0002C030010594000006C0300105003001046
:1040C000014B18607047C04638030010094B10B50B
:1040D0001A68191C084B002A03D1084C2468226076
:1040E00003E01A68904200DA101C186001230B608C
:1040F00010BDC046400300106403001038030010D8
:10410000034B1B68002B01D1024A13607047C04665
:104110004C03001040030010014B4A3318787047DD
:10412000CC04001038B5164B1A1C98321268002ABD
:1041300004D0144B1C6801231C4001E094331C681C
:10414000114DAB689C4202D16A68002A16D0002C3F
:1041500002D1002B0AD111E00C4B1B68002B02D0BE
:10416000201C6968984700236B6006E0074B1B68BA
:10417000002B02D0201C211C9847AC6038BDC046E3
:10418000CC04001048030010680C00105803001005
:10419000084B1860084B1960002809D0074A012312
:1041A0001370074A00211170064A9061064A137085
:1041B0007047C04654030010700300105C030010E9
:1041C00044030010680C0010300300102D4B73B531
:1041D0001A682D4B1168186881421BD0002100918C
:1041E000019112681A60294B1B688B4202D0684605
:1041F00001A99847264B00991C68181C019A254B69
:10420000A14202D11C68A24202D0234C0125257094
:1042100001601A60214E336A002B10D01E49002322
:10422000CB56002B2CD01E4B00229A56012A27D1A8
:1042300000220A701B490A7002221A7020E0144BF7
:10424000174C1868002807D00023E356002B03D131
:10425000104B1968FFF79CFF0023E356114D022B0A
:1042600003D100232B70B36123700023E356002B8E
:1042700002D00A20FFF72AFF0022AA560A4BDA666C
:1042800073BDC0463C0300100C0000106803001012
:10429000540300107003001044030010680C001059
:1042A000300300105C030010CC04001008B5084A6D
:1042B000084B126819688A1A05D5FA2252001A604A
:1042C000054B1A6801321A60FFF72CFF08BDC04683
:1042D000340300101400001048030010F8B50E1C41
:1042E0000E21041C171C00F0A5FF174B03259E424E
:1042F00011DD092363730123237323E0301C0A219A
:1043000000F08CFF301C61550A2100F031FF0135AF
:10431000061C0D2D01D0002EF0D1EF1B033F27709E
:104320006B1E022B05D0E15C621BD2185173013B5E
:10433000F7E70F235D1B013D6B1C032B02DD002300
:104340006355F8E7F8BDC046FFC99A3B37B5041C72
:104350000025002300930193124B1B68002B02D011
:10436000684601A9984700980135002800D000252B
:104370000220FBF7E4FF0C4B1A680C4B116818681D
:1043800081420AD012681A60FFF790FF002C04D017
:10439000013C002C01D1201C02E0032DD9DD0120BD
:1043A0003EBDC046680300103C03001060030010CF
:1043B0000278002A01D1802252004378002B01D1DB
:1043C00080235B00D01A7047F0B59B23234D5B0020
:1043D000EC5C85B003900E1C002C01D1802464009D
:1043E0003023FF33EB5C002B01D180235B00029371
:1043F0003823FF33EA5C80235B009C4203D00F2309
:10440000171C1F4000E007271548FFF7D1FF02994E
:10441000421C631A802149000C1B0721C91B009410
:10442000019103980F49FEF749FB002333704124A3
:10443000301CFEF794FBBA235B003718E818001B0A
:10444000FFF7B6FF221C031C0749381C0134FEF796
:1044500035FB462CECD105B0F0BDC046CC040010B5
:1044600000060010389B0000459B0000F0B5634D2E
:10447000634C2B1C94331B6893B0061C0F1CA0616B
:10448000E161002B17D118280BD1C32909D15D4B4D
:104490001B680F2B05D1281C38300E21162200F086
:1044A00033F9A069182804D1E269332A01D100F058
:1044B000D1F8FFF7B7FD002E02D00A23636100E0B8
:1044C0006661301C391CFFF763FE4F4E33681A6873
:1044D0004E4B1A60FFF714FE01232B6700201423B4
:1044E000009301904A4B1B68002B1AD0494E336849
:1044F000371C002B15D01B68002B04D1464B1B68C2
:1045000098473B68F7E733681A68013A1A60434AEC
:104510001368002B05DD013B1360002B01D1FFF771
:10452000EFFDFFF749FD002801DAFBF7C3FF3C4B25
:10453000019A9A4204D040239A433A4B9A420BD1B3
:10454000A36A394A934204D008229343374A9342DC
:1045500002D10A20FFF7BAFDA36A2E1C8C36019304
:10456000334A336893421AD0324A93420FD0324AC8
:10457000934223D1FFF7D6FDFBF710FF2F4BA0612D
:104580001860224B1A68013A1A602D4B15E02D4B2A
:104590001B68002B12D00120616898470EE02A4F5B
:1045A000386800280AD002A80AA9FFF70DFF3B6867
:1045B00002A80AA99847336827333360009E009AFF
:1045C000013E002A03DC214B14261B6898470E4B42
:1045D0001A681F4B11681868814206D012681A6069
:1045E000FFF764FE0C4B1B6898472A6F002A01D026
:1045F000009677E7FFF796FD13B0F0BDCC040010EE
:10460000680C0010100000103C0300100C0000109B
:1046100040030010380300106C0300106403001006
:104620006E02000026020000FB030000E30300000E
:104630003E2700005C280000790D000054030010A4
:104640007E0D00005803001074030010500300108A
:1046500060030010F7B5274E002033681C68FFF791
:1046600075FE33681A689442FCD01B6801272D330D
:10467000FF330193FFF7D6FC1F4C0A231F4D6361E4
:104680001823A3611523E3612B1C9033002267627A
:104690001A60FFF7C7FC2F673368019A1B689A42BC
:1046A0000CD0FFF789FC3268154B116818688142FD
:1046B000F2D012681A60FFF7F9FDEDE72B1C012715
:1046C0009033182000211E686762FFF7CFFE0D4B64
:1046D000301C196800F04CFD3835011C0422281CE0
:1046E000FFF7FCFD1823A3610023301C6762E36120
:1046F000FEBDC0463C030010680C0010CC04001046
:10470000600300103403001070B5002A10DD047837
:1047100001231C404B1E002B08DBC55CE4006E0827
:104720003443C4540124013B2C40F4E7013AECE744
:1047300070BD30B59A4205DC845C8D5C85548C5428
:104740000132F7E730BDF0B5069E051C07A80478D6
:104750003078002A17D0059EB34217DCCE5CD75CB8
:10476000F7193F180020A74201DB3F1B0120EF543F
:104770000133F0E7CA5C12180020A24201DB121BD1
:104780000120EA540133059A9342F3DD01231840D6
:10479000069B1870F0BDF7B50AAC2478099D00940B
:1047A000089E2C78002833D000292ED0002A1CD057
:1047B000B3424EDCCF5CD55C7F1B3F1B0024A7427D
:1047C00004DA009C3F190F2427400124C754013309
:1047D000EEE7CA5C121B0024551C04D1009C0F227A
:1047E000013C22400124C2540133B342F1DD30E0E8
:1047F000D15C4942091B0024A14204D0009F0F2430
:10480000C91921400124C1540133B342F0DD20E035
:10481000002914D0002A08D0B3421ADCCD5CD05C49
:104820000133281A041BE40FF6E7B34211DCCA5C1B
:104830000133141B013462425441E4B2F5E7B34240
:1048400007DCD15C013349420C1B611E8C41E4B290
:10485000F5E701231C40099B1C70F7BD70B5049C53
:104860000125257000290BD09A420BDC865C8D5CFB
:10487000AE4209D10132F7E7815C002904D101324F
:104880009A42F9DD0023237070BD914204DA431887
:104890005B7843540131F8E70023435470478A4260
:1048A00005DD8318013B1B788354013AF7E70023A9
:1048B00083547047F7B5134A134C13785278C35C8E
:1048C000134000D04023114923601231009100228F
:1048D0000023A6187360009B0125123B1F785978AE
:1048E000C75D394202D077682F437760009F02335B
:1048F0006D00BB42F2D1123304320093282AE7D173
:104900000020FEBD04010010280E00105000001011
:10491000122330B54B43334A0131D318052251439A
:104920001A785C78825C144204D02F4A5F245218B3
:10493000947054709A78DC78825C144204D02A4ACD
:104940007C245218533214701A795C79825C1442B8
:1049500004D0254A7C245218A33214709A79DC7949
:10496000825C144207D0204C5F226418251CA235BB
:10497000A1342A7022701A7A5C7A825C144204D0C4
:10498000194A7C245218A03214709A7ADC7A825C1C
:10499000144204D0144A7C245218503214701A7BEA
:1049A0005C7B825C144207D00F4C5F226418251C8C
:1049B000523551342A7022709A7BDC7B825C14421F
:1049C00004D0094A2E245218A43214701A7C5B7C3D
:1049D000825C134204D0044B5918F43127230B7026
:1049E000002030BD50000010980C0010F8B52E4D7E
:1049F000061C00272C1C281C20214F22FEF78CF8B7
:104A0000002F04D02A1C7C2339322B7013702B1CEE
:104A10004F33002201371A705035052FEBD1211C7E
:104A20002D2338310B70211C37310B70A121A3705D
:104A3000637049005F2363544221FF316354A32113
:104A400049006254194A11785278715C0A4204D0C4
:104A5000221C53325234137023700024211C301C4A
:104A60000134FFF755FF0A2CF8D10024104B114DEB
:104A7000E25C1B19B15C58780F4A6300084201D010
:104A8000D15805E0D058FEF76AF80C49091A0A31E6
:104A9000281C023400F0D8FB122CE7D1281C08494E
:104AA00000F0D2FB0520F8BD980C001004010010A6
:104AB00018000010D80D00102C0000100601001086
:104AC0004D9B0000F0B5944B87B003901F68FCF736
:104AD00005FC92490022924C02910192019B0C2507
:104AE0005D43002B00D101258B4B1968032903D0AE
:104AF000042900D13EE202E0884A029202E0022943
:104B000000DCAAE0002305AA537023687F2003403D
:104B10005B2B72D02CDC232B00D19AE014DC062B0B
:104B200050D006DC002B4BD0022B00D094E0492360
:104B300090E01C2B00D18AE0212B00D185E0072BCF
:104B400000D089E0372385E0402B6ED008DC392B7C
:104B50006FD03F2B67D0382B00D07DE04C2379E01D
:104B6000502B72D0542B74D04F2B75D1332371E05E
:104B7000732B68D012DC662B41D007DC5E2B5AD039
:104B8000622B64D05C2B67D14F2363E06F2B3CD04A
:104B9000712B54D06D2B5FD135235BE0792B4CD03A
:104BA00006DC762B4DD0772B41D0742B54D148E0C6
:104BB0007D2B26D07F2B26D07C2B4DD1422349E064
:104BC000202347E031231370019B022B00DCB8E166
:104BD000231C083B1B680340542B0AD0019903296E
:104BE00000D1AEE1231C0C3B1B681840542800D0B8
:104BF000A7E14C2205AB1A70A3E132232AE034234B
:104C000028E0362326E0382324E039231370019B63
:104C1000062B00DC95E1231F1B681840472323283F
:104C200000D08EE116E0302314E02D2312E0412362
:104C300010E043230EE044230CE045230AE0462322
:104C400008E0482306E0502304E0522302E0552305
:104C500000E04E23137074E1CF1E012F62D0022FAB
:104C600000D1E1E0002F00D03EE1226801231A428A
:104C700005D0A81CC0B2391C0522FCF7A7FB23688D
:104C80009B0706D5E81D0121C0B20A1C0323FCF7CF
:104C90009DFB21680423194205D0E81DC0B20521FF
:104CA0000122FCF793FB2268120706D5A81CC0B2AC
:104CB000092105220123FCF789FB2368DB0606D5C1
:104CC000681CC0B2052101220423FCF77FFB216888
:104CD000890606D5681C0121C0B20A1C0323FCF713
:104CE00075FB2268520606D5A81CC0B20421052215
:104CF0000123FCF76BFB23681B0607D5281C093032
:104D0000C0B2092102220123FCF760FB2168C9051A
:104D100000D4E9E0DCE0C04614010010C85B0000EC
:104D2000280E001022683A420ED0EEB2B01CC0B27B
:104D3000002105223B1C0336FCF748FBF0B2391C6E
:104D400003223B1CFCF742FB23680222134205D0DE
:104D5000A81DC0B201210323FCF738FB21680423FE
:104D6000194205D0A81DC0B205210222FCF72EFB76
:104D700022680826324211D0EBB2181C0230009390
:104D8000C0B2092105220123FCF720FB009B311C46
:104D90000333D8B203220123FCF718FB2168C906AC
:104DA00006D5681CC0B2052102220423FCF70EFBC5
:104DB0002268920606D5681CC0B201210222032394
:104DC000FCF704FB23685B060ED5EEB2B01CC0B244
:104DD0000421052201230336FCF7F8FAF0B205217D
:104DE00003220123FCF7F2FA2168090607D5281CE3
:104DF00009300222C0B20821131CFCF7E7FA22682E
:104E0000D20571D5EDB22E1C0A36F6B2301C08213F
:104E100002220323FCF7DAFA0935301C0B21FCF7D8
:104E2000C1FAE8B20B215DE02368DB0706D5681CF8
:104E3000C0B2002107223B1CFCF7C8FA21680222FD
:104E4000114205D0A81DC0B200210623FCF7BEFA0E
:104E5000226804210A4205D0A81DC0B202220623FE
:104E6000FCF7B4FA236808210B4205D0681CC0B2D5
:104E700007220223FCF7AAFA2168C90606D5681C96
:104E8000C0B2042102220623FCF7A0FA226892068F
:104E900006D5681CC0B2002102220623FCF796FA50
:104EA00023685B0606D5681CC0B2042107220223D2
:104EB000FCF78CFA2168090607D5281C0930022264
:104EC000C0B20821131CFCF781FA2268D2050BD569
:104ED000EDB2281C0930C0B20B210A35FCF762FA8A
:104EE000E8B20A21FCF75EFA019B04340133019316
:104EF0000B2B00D0F2E5214B1B68002B05D020487E
:104F0000002109221F4BFCF7D7FA1F4D0024023560
:104F1000AB1E1A7803996B1E8A5C1B78134208D06B
:104F20001A4BA200D0581A4B0922E15C154BFCF732
:104F3000C3FA01340235092CEAD1FCF7D9F907B0DC
:104F4000F0BD002205A8291C029BFCF7B5FA2268D7
:104F5000120605D5E91D0F480022029BFCF7ACFAAA
:104F60002168C905C0D5E91D0B480022029BFCF74A
:104F7000A3FAB9E7094B0293C4E5C0464401001007
:104F8000579B0000C05B00001800001018010010C3
:104F9000B09B0000B15C0000559B0000D05B00009E
:104FA00038B5FFF7B9F80624002805D1FCF7A0F9B9
:104FB00038BD01340E2CF9DC0321201C00F0D8F898
:104FC0000321C5B2201C00F029F9281CC9B2FCF746
:104FD000E9F9092CEDD10B24EEE7000038B5041CEB
:104FE000FFF768FC201CFFF76DFD094B1B78002BB9
:104FF0000DD0201CFFF7FAFC064CC8235B00E51817
:10500000211C05485034FDF74DFDAC42F8D138BDA8
:1050100080030010980C0010D753000000B589B031
:1050200000280ED0FCF725F901A80921FEF74CF95C
:10503000684612300A21FEF747F901A8FFF7CEFFB4
:1050400008E0FCF71EF9044B1B78002B02D0034844
:10505000FDF728FD09B000BD80030010599B00003A
:10506000FEE7FEE708B500230B4A0C499A188A426E
:1050700004D20B49C95C01331170F5E7094B0A4AA8
:10508000591C013B934203D200221A700B1CF6E715
:10509000FBF7B0FDFEE7C046000000103C01001029
:1050A000B99B00003D010010540E001002B471467F
:1050B00049084900095C49008E4402BC7047C0465B
:1050C00003B47146490840004900095A49008E441A
:1050D00003BC7047002934D00123002210B4884259
:1050E0002CD301242407A14204D2814202D2090117
:1050F0001B01F8E7E400A14204D2814202D2490038
:105100005B00F8E7884201D3401A1A434C08A042DA
:1051100002D3001B5C0822438C08A04202D3001B70
:105120009C082243CC08A04202D3001BDC08224387
:10513000002803D01B0901D00909E3E7101C10BCAB
:105140007047002801D00020C04307B4024802A1E4
:105150004018029003BDC046D90000000029F0D0DD
:1051600003B5FFF7B9FF0EBC4243891A1847C04682
:10517000002941D010B4041C4C40A4460123002255
:10518000002900D54942002800D5404288422CD34E
:1051900001242407A14204D2814202D209011B0149
:1051A000F8E7E400A14204D2814202D249005B0048
:1051B000F8E7884201D3401A1A434C08A04202D3B0
:1051C000001B5C0822438C08A04202D3001B9C08F1
:1051D0002243CC08A04202D3001BDC082243002853
:1051E00003D01B0901D00909E3E7101C6446002C19
:1051F00000D5404210BC7047002806D003DB0020D9
:10520000C043400801E08020000607B4024802A124
:105210004018029003BDC046190000000029EBD0E1
:1052200003B5FFF7A7FF0EBC4243891A1847C046D3
:105230007047C04642180023002903D00370013094
:105240009042FBD17047C04670B5061CB30717D11A
:1052500033680F480F4D1A189A43301C2A420FD159
:10526000043002680A4BD41894432C4208D104300D
:105270000268074BD41894432C42F1D000E001306F
:105280000278002AFBD1FDF773FC301C70BDC046CC
:10529000FFFEFEFE8080808025732025730D0A00AE
:1052A000444D31355F4D38300053455249414C2013
:1052B000434F4E534F4C45007265616479000D0AAF
:1052C0004279652E2E2E0D0A004E4F00203F0025FC
:1052D00073202573202025694D485A005632380026
:1052E000202025692E25303369560020257352541D
:1052F000432000444D343100444D3431204F4B00A5
:1053000020204552523A20256900424144204B4515
:1053100059202530327800202D2025303278004C5D
:1053200043443A25303269202D20256900505245EA
:10533000535320454E54455220544F205341564517
:105340000053495A453A256920555345443A256941
:1053500020465245453A256900535441434B3A0093
:1053600025633120484F5552002D0052544320529E
:10537000454144204641494C007475726E65642075
:105380006F6E003C52455345543E0D0A0042616425
:10539000206E756D6265722E0D0A004241543A20EE
:1053A00025696D560D0A000D0A253032782020003F
:1053B00057616974696E6720666F722064617461F9
:1053C0002E2E2E0D0A00426164206D6F64656C0DF7
:1053D0000A00526561642025730D0A004641494C5C
:1053E0004544006F6666004C4344206465627567FF
:1053F0002025730D0A00436F6E736F6C652074690E
:105400006D656F75742073657420746F2025692035
:105410006D696E757465730D0A00000000005C0014
:105420000C000C7C287C7C447C2410482854080008
:105430000C00384400443800201008103810804018
:1054400000101010004000201008384438007C0084
:105450006454484454281C107C4C54243854200470
:10546000740C28542808543800500080500010282C
:1054700044282828442810045408384C5C781478B0
:105480007C54283844447C44387C54447C1404388C
:1054900044347C107C007C0020403C7C106C7C40C0
:1054A000407C087C7C047C7C447C7C1408384478F8
:1054B0007C1468485424047C047C407C3C403C7C44
:1054C000207C6C106C1C601C64544C7C44000810E4
:1054D00020447C0008040880808004080078447818
:1054E0000007080400000000BF01BF01090500001B
:1054F00007000700070007130A00002000E400FC73
:10550000003F00E700FC003F002700040F080000F8
:105510000C011E01FF03FF032201E201C2190D006D
:10552000000E001F0011019101FF007E00FC00FE33
:105530000113011101F001E0140A0000EE00FF0167
:1055400011011101BF01EE00E0013001100105035E
:1055500000000F000F0A050000F800FE0307070116
:10556000040B060000000001040707FE03F80F0803
:10557000000000000A000E001F001F000E000A11AC
:10558000090000100010001000FE00FE00100010C6
:105590000010080400000004800780030D070000CD
:1055A000100010001000100010001008040000008F
:1055B00000800180010D07000C000FC003F0003CCB
:1055C000000F00030F080000FE00FF0101010101B0
:1055D0000101FF01FE10080000000002010201FFAE
:1055E00001FF0100010001100800008601C70161F0
:1055F00001210131011F010E010F0800008200830B
:1056000001110111011101FF01EE1109000030002B
:1056100038002C002600FF01FF012000200F0800A9
:105620000080009F011F0111011101F101E10F082C
:105630000000FC00FE010B0109010901F901F00F56
:1056400008000001000100C101F1013D000F00034D
:105650000F080000EE00FF01110111011101FF010F
:10566000EE0F0800001E003F0121012101A101FFF2
:10567000007E0804000000008C018C01080400007A
:1056800000048C078C0312090000200070005000F9
:10569000D80088008C0104010401110900004800B1
:1056A00048004800480048004800480048110900E8
:1056B00000040104018C018800D800500070002013
:1056C0000D07000002000300B101B9010F00061927
:1056D0000D0000F800FC010603FB06FD05050505AD
:1056E00005FD05FF050601FC01F812090000800117
:1056F000F0017C004F004F007C00F00180010F089A
:105700000000FF01FF01110111011F01FE01E01165
:105710000900007C00FE00830101010101010183F9
:10572000018211090000FF01FF01010101010101D6
:105730008301FE007C10080000FF01FF0111011130
:10574000011101110111010F080000FF01FF0111FA
:105750000011001100110001120900007C00FE0080
:105760008301010121012101E301E201120900008D
:10577000FF01FF011000100010001000FF01FF01E9
:105780000A0500000101FF01FF0101010B060001F4
:10579000000101010101FF01FF10080000FF01FFEE
:1057A0000138006C00C6008301010110080000FFF1
:1057B00001FF0100010001000100010001160B00C2
:1057C00000FF01FF010F003C00F000F0003C000F63
:1057D00000FF01FF0112090000FF01FF010F001C83
:1057E000007000E001FF01FF01130A00007C00FED1
:1057F0000083010101010101018301FE007C0F080A
:105800000000FF01FF012100210021003F001E14C4
:105810000A00007C00FE00830101010101010383F5
:1058200007FE047C0412090000FF01FF0121002192
:10583000007100DF008E010001110900008E009F41
:10584000011101110111011101F301E2110900001F
:10585000010001000100FF01FF0101000100011131
:105860000900007F00FF008001000100018001FFAE
:10587000007F1109000007001F007800E001E0012F
:1058800078001F0007190D00000F007F00F001E0F5
:10589000017C001F001F007C00E001F0017F000F71
:1058A000120900008301C7016C00380038006C0049
:1058B000C701830111090000010007001E00F80163
:1058C000F8011E00070001120900008101C10161F9
:1058D00001310119010D0107010301000404020057
:1058E000007F0109050000070000000000070B060B
:1058F0004400FF0144004400FF01440B0600008CFB
:10590000001201FF032201C40D078200450025009B
:10591000920048014401820C060000E600190126AD
:1059200001C000200107040000000001000208047B
:1059300000000000FE010102080400000000010256
:10594000FE010B0600008800500020005000880B6C
:1059500006000020002000F80020002006030000C0
:10596000000400020B0600002000200020002000A0
:10597000200603000000000001090500008001600E
:10598000001800060B060000FE00010101010101E4
:10599000FE0804000002000200FF010C0600008265
:1059A000014101210111010E010B060000820001DD
:1059B0000111011101EE0B060000600058004600C5
:1059C000FF01400B0600009F00090109010901F1D8
:1059D0000B060000FE00110111011101E20B06008F
:1059E000000100C10131000D00030B060000EE00B4
:1059F000110111011101EE0B0600008E00110111C1
:105A0000011101FE0804000000008C018C01080453
:105A100000000000000208010A05000020005000FC
:105A2000880004010B060000500050005000500098
:105A30005009050000040188005000200B060000FA
:105A400002000100610111000E0D0778008601328D
:105A5000014902390242027C0E07800170004C00AD
:105A600043004C00700080010B060000FF01110193
:105A700011011101EE0B06FE0001010101010101FE
:105A800001820B06FF0101010101010182007C0C72
:105A9000060000FF0111011101110101010B0600B7
:105AA00000FF01110011001100010C06FE000101B0
:105AB000010111019100F2010C06FF01100010001C
:105AC00010001000FF010804000000000000FF01AA
:105AD0000704C00000010001FF0E070000FF0118CD
:105AE0000024004200810000010C060000FF0100BC
:105AF000010001000100010E07FF010C003000C091
:105B00000030000C00FF010C06FF01060018002009
:105B100000C000FF010B06FE0001010101010101AF
:105B200001FE0B06FF0111001100110011000E0C07
:105B300006FE000101010141018101FE020C06FF88
:105B4000011100110011002900C6010B0600008E92
:105B500000110111011101E20B060000010001001A
:105B6000FF010100010B06FF000001000100010020
:105B700001FF0D0703001C006000800160001C0095
:105B8000030D071F00600080017C00800160001F82
:105B90000E07830144002800100028004400830100
:105BA0000D07030004000800F00108000400030EC4
:105BB00007810141012101110109010501030100D2
:105BC000030720611A5400000D0C205ADB58000016
:105BD0000D0C205AE054000000070008000A0100E4
:105BE000181110133831303378717073C8C1C0C3C5
:105BF0008881808384848782C5C4C7C275747772A4
:105C00003534373215141712020702080201000357
:105C10000109030402040205030500062024282CC0
:105C2000383C4044484C4669726D77617265202566
:105C3000735F5632380D0A00252D313073202573DD
:105C40002573000D0A5479706520273C636F6D6DD4
:105C5000616E643E203F2720666F72207061726122
:105C60006D730D0A00557074696D65202575730D8F
:105C70000A0025730D0A0D0A00564F594147455237
:105C8000203E3E200025630048656C70004E6F206A
:105C9000706172616D73004B65792070726573730A
:105CA000003C6B6579313E203C6B6579323E202E9D
:105CB0002E2E0044756D70206D656D6F7279004CED
:105CC0006F6164206D656D6F727900637400436F5E
:105CD0006E736F6C652074696D656F7574003C6DD3
:105CE000696E757465733E004765742074696D65EF
:105CF000007473005365742074696D65003C5959D4
:105D000059594D4D44443E203C48484D4D53533E17
:105D1000007464005570646174652074696D650079
:105D20003C6F66667365745F696E5F6D696E7574EE
:105D300065733E00546F67676C6520646973706CAF
:105D40006179206F757470757420746F20636F6E45
:105D5000736F6C65006200526561642062617474E7
:105D600065727920766F6C7461676500CD520000B2
:105D700000000000E91B0000885C00008D5C000052
:105D80008B5C0000FF000000B9100000975C000071
:105D9000A15C0000E95E000000000000DD0E0000D4
:105DA000B35C00008D5C0000775E00000000000026
:105DB0007D0F0000BF5C00008D5C0000CB5C00002C
:105DC000010000003D110000CE5C0000DE5C000020
:105DD000CC5C000000000000050E0000E85C000044
:105DE0008D5C0000F15C000002000000650E000008
:105DF000F45C0000FD5C0000115D0000010000008B
:105E0000A50E0000145D0000205D0000125D000082
:105E10000000000011110000345D00008D5C0000E6
:105E2000555D000000000000F10D0000575D00000E
:105E30008D5C000000800150008002500080035003
:105E4000FC3F0150FC3F0250FC3F03502578000D01
:105E50000A413A2000202025633A20000D0A533AD7
:105E600020000D0A4D3A20002020473A20253032EC
:105E7000780D0A006661696C00253034692D253083
:105E800032692D2530326920253032693A25303289
:105E9000693A2530326920257300253032783A2559
:105EA0003032783A253032692E253032690025307B
:105EB0003278203A202569202569203A2025303281
:105EC00078004E4F2052544300253032783A253026
:105ED00032783A2530327800253034782D2530322A
:105EE000782D253032782020257300000C5F0000CB
:105EF000105F0000145F0000185F00001C5F0000CE
:105F0000205F0000245F0000785C00004D4F4E00D1
:105F100054554500574544005448550046524900E1
:105F20005341540053554E00CCC5ED2D1207EE766B
:105F3000A609CFA6C6FC205FFD8D1416A5B8757AFC
:105F40003E3979BAAC30388E4526243C71EA4D1D75
:105F5000FC6918F8374D202D5431210C7B81EFB9A5
:105F60008C658A36C3DF9BAF1E308AD6E807680B84
:105F70000BE035688B58BB367E32A97A0BFA57FD99
:105F80000296BF98D0985FEC4861E9BA233F67B9A1
:105F900033A85C1D8A2E7C20E734A69E180B6385EF
:105FA00021022479A02300408133DC942FFB993C0B
:105FB0005492B0BE5BC9D31C43B1DDD882327602A5
:105FC000251407C50DB09AA840A8A51E3236A06AB0
:105FD000EE5A06EA4519FB4815D28106CCA266485E
:105FE00045065893AC0C6D5B5B16F4E389E8A45F3F
:105FF000A5CC5CE2F9AC69CE6D5B587537C847AB90
:10600000C306D05F490DF7D3728C03EE6C76DFD4F4
:1060100000858D59558EDC03D6F46B0DECD3879C2F
:10602000B706E117A13110ECD4887F1F10CA9FC2B8
:106030003E76045EA638315A0F1949812919BDDE12
:1060400016F74461A154A2E5ED29ADA66BBA4C0B3D
:10605000B86D36E573F542257B305B05AE43AA95F6
:1060600062856B34907EA481B93B4366448372524F
:10607000D0B598FB7C73D92076A23A827F51C22793
:106080004FDC7FBB8A9ACD3FBD4DDBE778C92198B5
:106090003DCD24CD2698FB0B4161E9A65592AE9DDE
:1060A000C6A681AAC9E86FCA34249BA239A331903D
:1060B00056AC2FFE5593AB5EAFDBAC7A01AF54C349
:1060C00074119848048C2DB6A1A94451730AD9D9EA
:1060D00045AD4153EDEFC9086455FF4CA4382A592A
:1060E0005B084DCBD85EE3F04527E204E16D1CBEB2
:1060F000F4C273E99F818CF866229A6D0C32D98BB9
:10610000088E4F8419611A2FC61CFC225919B1350B
:1061100050CADEB8B48E39C58652776910C4E31907
:10612000A4391728409DE89C34CDE74EFDA3AB571A
:106130001ACDE49B6787A4D6975534F9F710871BCF
:106140006628B1090B342D9697B2EE0A76879DEF3B
:10615000C602940373943DD9D2F69ABD50E96EA657
:10616000D70ABAFCBC8E6E45B0AFC5DDD821FF445E
:106170008AEF678FD6D734C920A68C6DC459CD6CF1
:106180006D5171B1691A45A79C15BB56A10CF2312E
:106190008E1A0411C7EED93DCA1EEF4DE5F968A36A
:1061A000B5D55CC5C16A188675FA25D704F0BE5D01
:1061B00087DB9EF9F97A663955162C8B8DC9A8DED6
:1061C0007C1E956DF86C514F29CA4820B8C0DC4D33
:1061D00072A4F7ACA54A4DED02DE7E4E9E8727BD28
:1061E000C8F7A2658A4FE9ECE338336F6BB7B8ACF8
:1061F0009AA5FD068DE255B7BD0D51CADBF62049C3
:106200000882928C113F4632852BBC13E8B2B557F9
:10621000CDD73C090B6F55A3BA423D2BE47A8C765F
:106220009718A79840096154979F9313418D0E5A70
:106230001D57932772739799AEC133EF4604FB4005
:106240002A8991186AF0D8C200D6DAD984DCCEAC9B
:10625000B8379BFFA463D0F25F862682331593FA8A
:1062600087F931DD495CB55DAA46C9A7D3C5A3CA84
:10627000C2735E9E8018CD4C2D6B9ED6C325B13661
:106280005C49024F0FF606057FC5E755C164E81962
:106290005A8C5C4C9C441008BAC6DF9CBEC942BBF9
:1062A000D760993A18DFEA19268E6A5996F40D34A8
:1062B000747F4D88A93DF8F0BD47D88FCF48814AFB
:1062C000793F42D30B3E4CD3376D49F1DCD5990968
:1062D000198CF57D6F5688B98AAC2246751DB5B606
:1062E000DD07FC115E295A04A40861B492D6211777
:1062F000D06BD871719BE3A4D0A5C4E5F091CEC357
:1063000057A5A372F926EABE6A72FF82447D6E0920
:10631000FC643D54AC8B607D5107216781A1FDEF8A
:10632000EDF97896CA84E72BA8BD656900AEA6C0D2
:106330008BF25EF5D21A1C5E6B2D87E1EB4331A028
:10634000E997540A55920BC633B8DEE4C2451C8661
:10635000EF3B9B8D38A25BF5A2EDDE55A4EC8A18CD
:10636000EBD67D26EB364049A1FAACC50DC5FC8BBA
:106370009D077F22F38D36ADE521A2A4BA103DA979
:10638000DE017D1A8C23388B40BBD773814AC54F01
:1063900036E87A4D2E50510297C1F17E4BB852B477
:1063A000A196006A8E8BE47803D5E2DC39170B3EA8
:1063B0009084B824B2A9F11D3957D43715BD754260
:1063C00090AD8BD8BE099505E7FAE5B1C667D7B1A0
:1063D00091BC1ED46A671C2421EBAE6AD89143F3AA
:1063E000E317B6E4B0630AF6BE016F16FF8EB9BFBD
:1063F000B3723A54A98E35FD033FBB9ECA6FA48B7E
:10640000C3F343F5A07EA4DCFD2761C11C0CE16A47
:106410007F2CA21A3583B9517A9F471D14855E845B
:10642000E39F79513CE363398D718F61DAEA225140
:10643000E7A255A199F1EA8986939C2B52DC0E893B
:10644000DCE2862C8749E4B88F223F907DE7EF3667
:106450009B12BE3D57610D255CD43CEE9E28859E67
:106460006278FDD97E4C5942253167A542157D30B1
:10647000B2039A0D26E01A303EF2016FFA98F1202D
:106480001524F10C877B59DBCAC16B9706164EC7E2
:10649000C61E1E958EEC8987092D343A0056B5C666
:1064A000558F2B6456D5933D758618553053362736
:1064B000CCC5E4CD05822759FF5FC0531407A7DF81
:1064C00057CC3208DD665203718EE0048E78A02F1F
:1064D0002BDCD8302427DE6822FA86172E2690245B
:1064E00034CD9ABAF7BE64D7E68B3749A3E2905C05
:1064F000798382609D4A1F0CC099460263AE72E1A7
:106500000F9472FB1BC17363F6E2D93096439D0E64
:106510003D180A672762FCC95BB0C26308C0AA8F36
:1065200051E44A4DEC6FF3CA22371E91ADA047E803
:10653000BDE8EB903DB1B0452B4F021C4FFD5C1800
:10654000A8B35EA7BE55D5B98568EA58E8F308BF79
:1065500002B226559E96F0282C300A3CDD13AE90F0
:10656000D83C5A1CB90C1494B1AD7112B8902339AF
:10657000F4B68D4D200E15607FDC8138D2E58A851A
:10658000AFC1A8EF2D0BAC92344346E9718546AFFD
:1065900020B3EB0E3AC8332392D1C0F51F4EEE0C58
:1065A00054B6FBDBD4FFF4C3755A06291518B8EEB0
:1065B000E93A52F2DB370C7BB332FFE0EC03A85729
:1065C000E58FB6CBBD9377500DEA3EE7FDF697AF6A
:1065D0004E1394C31B5426E1914FCEEB43E9997CB3
:1065E0008E4AC28DD6C2EBCFF311765AA26BF083DE
:1065F000EBAAC386858A744DAC32B1766C981BEEDB
:106600007C1B5E7A31A29D8164A0FF211A43C92EB2
:1066100056E2155BD51DF426143E0CB18AE207A4A0
:1066200077861D0D061177E95B10FC2FE4B58C0B06
:106630006C676FEB26C2F7662E4F8D82E5D6F16C44
:10664000A2450A64EA07590A7D81B8DB5B3DF5097A
:1066500043043C67CA4019131694F7A5B694D07C3E
:1066600096186B4674BA8BAD36AB2A98A2FB6F4274
:10667000B1F42D034AECB88727BF95B92BE53197C4
:10668000A16990C25145CB2F0FF4313BEB232E0C67
:1066900058CC507E1A13FAC6524ED1D46A417B04AC
:1066A0008FF176BE8F0068128C5FAECE046B19D16D
:1066B000DE1068718B65A472F36D5784586169DFD1
:1066C0002787A014E6EDEFCD94AF72A7FB6CD6E858
:1066D0006220B90676DFA9DE3071AFBA000E8256AD
:1066E0000F9C9476484DAB9CB87B47A5A7758FCC83
:1066F00073C5D4E393E02DBB872A37D4A282768F6B
:10670000FF915B5ACEBCF4BEA5B6107B52FB43B0E2
:106710002E8F1EF5F8215A573C0A7F2BAF5227BD0A
:1067200064283C5C052235D7F09B836460D0A1A42B
:10673000AE857E15ACE3EAFCF3317B8565243BC76F
:106740001EB41D406DC326C6F0FE240DEFDA6010A6
:106750008B9FB70B989A9DA84FE131F45E1BBA3717
:10676000B4E15A8D94A77E6167AD49D07124513B45
:1067700016F9057530762087EEFAF4DC65C7315FCF
:1067800019064602CDA58779DADCFE3C5AB1408075
:10679000EA4132C816CC97992545BFB22F70B3A4F1
:1067A000683E5BB591B13DADE7182B34B446AE5CA5
:1067B000B6ABC5997195BA5C5762198081E27CCEFF
:1067C000BD8C12622B2AC00A40A61AEE79F06BF635
:1067D0009B2F393EA7E643894B6233B4DFB0DD9887
:1067E0003DB0A0F60C502238708E9FA7251AEE45BA
:1067F00043E7C36F56BF1548704B6D9E9599C822ED
:1068000069D6283878095EB7F6AB9C80DDC82E3291
:10681000A4389CFBE2E22DB5B75D9C1D9C99DF9AE4
:10682000061CD8E6B3C7802A99C97F7311A83138EE
:10683000A0CCD322E7C41621508976133010BCFABD
:10684000861B2990FBF0EB4784A67DE096BDF7718F
:1068500037C91B9F45F1312410B105083474342524
:1068600035D17CAE6695698A315CEC1D82F729E5ED
:106870007F93CB24B687B96980A6987FB8676C8E62
:106880007CDC9B395C921988ABB8EE3621B1924022
:10689000CAFC813958F0F9654EDBBCCED225B7B4BD
:1068A0007DC0315051B1C8B5BFE321C02E8304175C
:1068B0006068A78D363618152BC28BB79E3BD19FCB
:1068C000BB8B7506281C6635C6A37D66B00E3A22C2
:1068D0008B7D57446CDA241A0E569D148F6B18D397
:1068E00003FD168601A00055D043329A4E0933A508
:1068F00006265689D49DE5C82F13DAC232A8FDBFFB
:10690000D65944420FFD93C0DFBA67B931633C8763
:10691000C4CA972C719BFA3A5256E00AD00EE94D40
:10692000748E454345913410EC348619B58563FF68
:10693000B8755CD67577ADDCA60C07210767DE6EEF
:10694000BEC49368B3275606351822CBE4686E4A56
:10695000597BECD0A2A7023521C72FA309D47B26EF
:10696000D5A9898DE5FD5AA948CAD40D23A016A939
:10697000F90AB56B49F6589FCFDA88C44616C0DFCE
:10698000F24B159B84BB90198322CA497D6C503011
:10699000E3A9CCEE2BE772086F2994860C1106351B
:1069A0001281A54813CE270C9281370B884F44895A
:1069B000702E69A8D116703B2D76A8F9D44FBB9ED6
:1069C000841558F89D363B6E68C9627DC38A75127E
:1069D0000419A65A77A3476A6C660CF175113F1922
:1069E0007A6A260F8A474E369D7E3E439AF3CDF74C
:1069F00095615D7A9B1DD97B3C97A4FD5C8C549975
:106A00004A18D2683982359F13201E93D05DAB118E
:106A1000D69AFDAC0B69F4AC1E5D7E0D82E59D77C8
:106A2000BED085CC936EDFD7BE8B367C9F04739E21
:106A3000E9875B58A8D8822861D9C105761212E689
:106A400062F735F5FA1911D53165DB48F9C4A5C8E7
:106A5000FE76EFE17461220A35ABC5E6B13DE74E43
:106A6000BB1BC0D330247C3E5049ECA51D4387BBE3
:106A700097DEB34FD8415ADDD366D571BB9D062D45
:106A8000750BB76C3C0FE76003BF3BBEBD3C178284
:106A9000EE4C524AD9FB66FE48862CC9F8BFF84432
:106AA00040F867D795517B7A970596C1F7E9C1F50C
:106AB000B9F3D6F78A9EBB97E8B03619EAD6FDCE71
:106AC000F7A8B6960A1E97A9FF5B78D5054F4364D1
:106AD0005C94A4311A2C42BCAD47FA7BB0B7FB1CC6
:106AE000FFBBD5C7FE4DB84B1C02E8191364BA0AA8
:106AF000E18F003010E32F57038D7E9B79A3055C57
:106B00001AE8B600C5EF06E0A073E444BBB5EE5E3C
:106B10001C58954B033EDD4298756796EB2B13C8C6
:106B2000303B5916CDC9F260E82A8E0DCC847988A5
:106B300004EE306EC923B8C493D8B4B1AF09611C58
:106B400020CB7FB5B8685E3DC0EC772042C4D6C587
:106B5000BC8B5F7114405B6AB9B3D75B6BC0D0214B
:106B6000CDD8A55F446EB28E8AEC76F38B0EDE8BA9
:106B700068A8EB608B0B65E7711EE0B62BCCC27486
:106B8000685ED81F628CC85FFD776FD855DC56FDF4
:106B90001F6FBB153AF11DA3F0575318C681E10AC8
:106BA000B9929EF5B8D9C7FEE37A255BB14E259719
:106BB00023D1C4C07A542EE9FA070C584243D715A2
:106BC000BA30A4BF387DB60A99A22EA12F25FB01A9
:106BD000C6E97D00A6A71F355A0DAF6BC9CC23327D
:106BE000BF95099E77E799A515FE56041D81FFED17
:106BF000E66E3171944AEEBCC0E6DEDC5405C33A61
:106C00004EC2A88481DC7065779D063CAC7BE08336
:106C100090CB19C70862DCC51DDFB814C1C8CC030E
:106C2000466601479A39CB4525D15AC9CEB73AE8CD
:106C30006EDC0AE57B307743F71606F8D3E64F4C57
:106C4000BCE02E4681B3D7C518E7CF36C26F85AEFC
:106C5000788A6854B77F8B3E4FC96A7477586F0B38
:106C60006F7E02D050D9371784C163ED039DB88081
:106C70004512FF762551A44ED1F32939AE1D9BD97B
:106C800060039FDCD0960829E08ECB494AF17EE173
:106C90004323E7321DEAB56C243771F7885662E862
:106CA0003F88B2C40962704A3F4E85239F84F97CB5
:106CB000A58691D6A9E085D94A0067F354E322FF5F
:106CC000C8D159978143A9C9674AE467091ECEE92B
:106CD000B8D417EE2B36A98038A5A469B5D6B2DC96
:106CE0000C3667A8A6FC3687513E8ACE82386C1CCB
:106CF0004129EE5D047B0A020D035AC109B703AFB7
:106D0000D651921D9858C3130A06EEDCA82A906744
:106D1000B746B74649854A7B3EFB601DC88D577C08
:106D2000BB881610AA441576FAC00653A245A3B133
:106D300067CE6EBF36D65E46CD3EBA3AA92486519E
:106D40003D0EF7F9F74767F0ABE5214D2150994229
:106D50001E88A5B365F970618902562222F63BDED2
:106D6000AA7B9279B0C85E2F500B9D792E0ED8B5B4
:106D7000307D81FF0267342D7436BBCFE344C3FE00
:106D80001BC3339649C43746976D6859DD8A1DDAAF
:106D90008D0A65CE0B28ACBF187E9BACC196A09324
:106DA000DE6053814734C47BEDD0842E810B101BF1
:106DB0004869C5051BAC690890E9F8C0FBA81AF73B
:106DC0006B623CB508E11379D055C1FC521FC81C59
:106DD000860C7A7632255630629C43A33641AE9BB0
:106DE0008E5F5313970DFC2BB83EC953815D3E5DFA
:106DF000E8B372D7771E14B35F2E659A29268A7975
:106E000060FFF38E6E1408465354A58847B6ADE86C
:106E100001A8ADACE803B2AF431157AA4848CC90E3
:106E2000CED0D6D0FEDA9760D72BDDDE85E934836D
:106E300086622D717512781E2140DF8C35ABA83823
:106E4000EE6F78CF9A313E2F3D6327EBE3F829D1DF
:106E5000675C52CEC52F9A1BB60849A94FB37F7CF9
:106E6000D4ED77257A31C0C4E1BA86C9A675294721
:106E7000F5C55CF69219248E43200B1729C8C92A40
:106E8000B1280E9659A5D034640DCACADFFC473923
:106E90009285F75DB86291A6D0838997A1BD1A6BE0
:106EA000A52890BC86596BAA1EE72B42DDB32F287C
:106EB000B5A6AE626DACC987C9323E3CB3727C697F
:106EC00060EB684DFBD21915DFD965557FAFBA0E5F
:106ED0005D733E0578433D75DF1FA2135DBFBB8523
:106EE0003D6C73EF59969F677EB81CF9CA8FE50118
:106EF0006EC25F49A124A775E1F6B184F6BA49AF25
:106F0000822C4901A235C8CAE7CCA10C5B9BE0FAF0
:106F10008576A1AB6599B8664AF14FEA5C01B47613
:106F2000D8462732C79E19AE4DFE616FDA939A6636
:106F30004BC9CF78AC79F88829D4FF40890B729679
:106F4000AAEAB4192130FBCA796C8A8957E7A8D814
:106F500027DEB2CA2EF963599665CFC1D86E726E1C
:106F6000240AB8D5B1B0958F58A063830B58196423
:106F7000CB06224C4E013554E7FBE349AF35BC69E3
:106F8000A10D48B58B0831FD2C2AE65896D88E8184
:106F90006DE61CAA75EED5E31C04B416EC027C6009
:106FA0007945C321D060A3FF576BCD5EA0B13DC230
:106FB00028AF46995D6D43D124946673B967624FDB
:106FC000CEA5991742196FF117222D6BE6D58605CC
:106FD000DC29662528BED963E10847BCCF8B18A9F8
:106FE000A14FE0E3981D62390AAF22E802298D180B
:106FF0001C5A8BA48AF6EE17A966E1AEAC7EA6AA4F
:107000006A723CC9F76950BEF9FA197E63D069FE0D
:10701000B0F351BC7ED9F1E3A8A0E862CD1064734F
:1070200077548714FBB4594BD72813742C7B31C881
:107030005E0978A56025E705A2F0DED4A2D696B950
:1070400063989C76C390374575B60D0B7027FC9DF1
:107050009C8B8FC609023FAE57F0929301576E6C1E
:10706000E542F7BA0100010DF1C8B70D4E5866C2EE
:107070003D6DDEB1F4AC0680234B1FDEA8A066B9DF
:107080007D87184D8AF5608D29A43941076D8139B6
:107090009A1F5D780A0FEF15EA843C7753FF1D0DA8
:1070A000755737F25C27B386FF7F3D24AB2F4ED652
:1070B000563611383579F65947A1C0C58B41CC9960
:1070C00045F3792E85AA5FE7D7389A3393E199E99A
:1070D0002CA908B602117B28861649CBE98A9F5253
:1070E00066C27E6FA997AEB1ADDA70F3BEE2573BD0
:1070F0008F73FDFA81796951F7CEAE782BB25FFFBD
:10710000518B24536EA927435C1376470784B9B08B
:107110002F1BCEA5885E4D16156A753F6EA947D107
:107120009745AA7563C42239C71F5F00E7F5D2A847
:10713000928A76FCBEA2469C95654940A390672A38
:107140003E26DFB33C4306A117E16548980A593053
:107150000041600B2B187CC415DCC5837841B6A4B4
:10716000BA26BE871AD986E0D43D3E98684FECCB4C
:107170003B2D1366358024EE98362FC0BC568DC249
:10718000DDC6CC96B0CD704BE6A75D86B04D1768D6
:107190006A139CBE8786AAE082625310DD98F7FDD1
:1071A000EE496CC9818F5E63465449F2655DCB86BA
:1071B00029A1CC1CB47799AC99D4431311B2911A7C
:1071C0004B092F91C007C96BD4C92E060C522DAFA5
:1071D0009A9A6D12AF00C654B59DB74331FCC35E99
:1071E000EF930B8E46F2272AD37C111365B345C962
:1071F0009282E092FC4009A6C7B2495A962D6AF1E4
:10720000C401619C771B92EB8440A9124EF063C4C9
:107210002B6D6DE056BBE315C3B8C329345C27EE74
:10722000F64EF29E0131C04A91C2BB945DEA0BE07A
:10723000C60D5CBA5ECC2C8D129C40F5EE875826AC
:107240009AC1252B214D9A72D14ABF0C1877E35869
:10725000ECFA6FFDB71D32A34F4128118144038022
:1072600075E538B1D939FDB7C72FEFF2187D4EEE6D
:10727000C48BEC8D5BAE1FF23ECE4A02114DE1B4E1
:10728000B16A79C3E997F1E24FDC8059A0148AE32F
:1072900049B140E52B774EC4F844FE4975BD3EBF69
:1072A0006D6DEBF8EDAB6BC09524FCB7EA65C607D6
:1072B000E58F177490163C5393BD9B0A4F122CBD5B
:1072C000C415B1D307B30742D8F4FF9983A5AC85A1
:1072D0001126263CA9442F16A37F778603BD60F0B4
:1072E00002EA89424F7DA4A13A5CABCDC110FE37C2
:1072F000BEC58C90531732B30CFA0FBEFE6241BB71
:10730000E514F1793A38E84C7DEEA65E9BF1449D98
:1073100094957D74C62D3FA85238076F7A6DBDD302
:10732000CF8FA7DF7BF064873DC73FFA358759EDE4
:107330009D04A7B00FB3B9495B692DF031D1C80ED8
:1073400036BFB606BC028929B47DFD1F4B81D08EA5
:107350001335C8AB66B2E027A6E4656939A21112FD
:107360002777A57BB770D8658F28F08EA9C9A5C3EC
:107370009432335DB834168DCE438FA00CC410F612
:10738000DBEF8EBE15D4C893A6DA077FE5C1A7BA96
:107390002F736F636C6721162389AE294291942560
:1073A00077CB78B9FFEBD61BA8D2FAB5B157C06539
:1073B000E58433F2A411BBA7F33569C7AE7FE714A8
:1073C0004EB40A7D2BFB84A89010A664887AB71768
:1073D000A0D74CE2940EC6EA46D9B8D780F1A400F3
:1073E00006837512CCB7AA5B7F367DF7A2F8D03141
:1073F0001E22BCDBF212AF40FD9D8154FFA3D136AB
:10740000CFCA71EFFFD2B8F9C62DBD4C827127A447
:1074100002890E895FBFED13D54EF80AC0C97F5EA1
:107420003A522DB38648907F04E2A694779FF42BBE
:10743000BD1A4F966A86BC383376EF9BF8660B947C
:10744000A3BFCFC651273DB307C787D760F368EC0A
:10745000019D8BAC0E6FDF48DEE0A43C0681283C2A
:10746000165EC6659DA69FA7B0CD58F112FE553594
:107470004DF4A6A6E8691D454D72AB682AA79A7C13
:10748000468A6DF906D296E6A7A7672BDFB9F6C143
:107490007083A3C7AED3A75104A834E0662AB00115
:1074A000E5F6CBAA2A374BFBB40403742FD745610A
:1074B00005A917369CC58A7AAEEE22C4422F1A8DD2
:1074C0005B3DA7E2DC75FDF59DB6053439EA8C62BB
:1074D0004EC85DDCBC0F9CDA318497A6B3DB3B1A47
:1074E0009F4DFC88958CFEF2D71A4F5AB3ECBCAE78
:1074F000AC374D56F3F4A56B493843A838EAA0875A
:107500002C34718238CE046BDB26DEDC161FF28B46
:1075100051693EDA444670C13BB4BA7E36AE1A9821
:10752000FB1657D3C2EDDE40FDAA541FFE0000013A
:107530003A8B56B79299641F2BD4E8EE1658008107
:107540002E2A739B94857188077E03A0026F5125B4
:1075500035AC34D6448193E50995C9E3D008E82BCE
:10756000A0E663021BD739B4227842AD2C41C5EBAB
:10757000A21C3715015B048A97E788871DC78FF91E
:1075800021D30BAC24B0446B310FB54E40A90DD9BB
:10759000124035570B4C0B4D1619672830C5775ED6
:1075A00042EF75C810A76AD79E6EDC2FD95BAA1070
:1075B0006AB2670EAAF235E2353DE67624AEB10234
:1075C000A87449E59DA9C831D09F4849CF8434E1CA
:1075D000F869CC67170A97112FAFF54A2DF94BBA06
:1075E000E8AB6C56EB45C93A90F7CFF35A6A084FAF
:1075F000CDA7CC0050BC06496263D372CB76E4269B
:10760000D308959C94D824B082913F3C179300F8FE
:10761000DA3929C0843D708FC3D12B4FD4BA1FF4FF
:107620007793EBD1F8FEF49828A68A6A0258933D26
:10763000308A0E41334127750E4DC72709049E1B22
:1076400025A77CA9EB65491BD35B267090612B9C19
:10765000CCBA820AFF1BB65B89FAB8EB2457B25D3D
:1076600080CAB786E6196395D4868773FDA0B5DD19
:10767000CCF3389EA61EC6F0800BFBEF0163FF70B3
:10768000FB86BD946BD8C55024302AAE7D301629B8
:1076900045C19D7D1C4BF9C784B8C5B9E2C70CC272
:1076A0000B94E9170BD131C0C18020CCE7A69DB067
:1076B0009CB5C6264F593C6BAA60F772FC66AE6754
:1076C0004E89248A229A2DD888B7B893BD82EF7349
:1076D00073DD44E8F4CB7F7066C6D6E6ECD30A4C83
:1076E00026DF212DBBF2DE689E8EBCCC6F30983B2E
:1076F0002A0F4CAD8109F55D8833323357828618E5
:10770000445ECBB1FFE54C03CF8BC447D0509ED82D
:10771000568436B4FE7A4450B57C0DCB0F45870EA7
:107720009FF2154A89C7FF03F143DD2C417157A031
:107730006139B507E479834B2E370339BD17B0F9AA
:10774000982D51635DD5D1B11FED015244C5E314AD
:107750002F156C368622D3D13BDEE795F9C73F1F44
:1077600030264B4818BF10A2EF0E5726E9127C5D59
:10777000FE95B7881A5F5BAA6DA5C801B68F2C303D
:10778000D8655F487D3A63D44C2AE91BC22F7F62DB
:10779000A7DBAF984CC412D515593796E867475CFC
:1077A00066354103DD33426F6C73181DA7636B842C
:1077B000D2E86BB3B64359F36231C3E580EB9E77F1
:1077C000C71285CEDA5E9B5C7157565E07DEBDA799
:1077D000DA9B959B5E7C68ACFD9AAD123AD4818BA6
:1077E0006834465F9236AF4C0EF35508B5F0FAF4A4
:1077F0007BB877095448EBEA9A62476F8D3DC26ABD
:10780000FD69D11E951B0F84EAA68311406E4611B7
:10781000B9FDB49F759566EB04EC22389BDFC4FB81
:10782000E15F1D793B3CAE19F4517AE39323293093
:1078300057AAE937E9D7EB9BDC45E92DF47786FFBA
:107840001DD71B3B67BEC7FDE1928E46E98064E60B
:10785000B062ED0347B63D19D95DBC629C0819447E
:107860003BFB558AF838431A374FA1646D2A41FA19
:107870005115478A5019CC358F4869AE1F55EE24F3
:10788000BC1C75DA9804F318CFB4E5BC9241D43629
:1078900015D504989D5EC91769C01E8689C4896084
:1078A000570669B0D0F5B0289F60B811447B5742A5
:1078B000A39CBA515EAE2EC4D35FAB5BED4908DC2E
:1078C0000CBECF4F9CD436B27AA2660A6DF3A28D5D
:1078D0007B5E28C9B49C962C88D9D95B2F48566901
:1078E000DF1C64C3C2E6631E93D3F08F121AC6D1A5
:1078F000BF84EB2B2CC1F94ED0C3401BF5736685BA
:10790000848D690D4A556BD80BA1D1A49E6A5D2F59
:107910000DFA765DE6539229751B59F92E99DDB65D
:1079200059C23ACF4126A2A3891A8548957B6EBFDA
:10793000F3CE95513B3F3DB3E0A5D3C0A84647B831
:10794000F3FCD04CCA6F773BDA4D7BFBD4FE1904B5
:10795000B2AF3660018548B012BC3D8556E2DF0902
:107960006D829CB859AF0CADBE89FF1C7B1F96770A
:107970007BEBF48CEA0271D56C04EA3DEAD8944BB7
:10798000FDB66B61C66A1D1809F95850F23A6CF2DF
:107990004E2A9EC1AB517C3F62655D7E8F5071E087
:1079A000F70C5AEA93AA988610D084F6C588F2D0CC
:1079B0004F4F5A529A0FE1E0A74ABC173665981DFF
:1079C0000B03EE2301CFFC31BD864D0D8A82C6FF2D
:1079D00067207BF8565889A127BEDE934BEC506791
:1079E000D6AA81F3C47A1002E485DBDA2CB9FFED64
:1079F00016D9EAA7CF9DBB700234E13A73198022F1
:107A0000F3B166C3E09D98369DB668C52A4ABACCE4
:107A100024E467A1868C9C3CD6FDE6C17B7CFF0AF2
:107A2000B9552E8E31D5067E1199E34A512DEC6061
:107A30003938DB493FBBD43FE400DA3E74B807F97C
:107A40005C7E111B433C2776A415ECA0B2DF69FADB
:107A50006B992251462EF396AD4F7AACB8B4B6630B
:107A60004320720C31258CFE1E3079EE655B276455
:107A700029F36A1FD07B7C820D36B68C9E71D56649
:107A8000F39BBE43D98FE4BBD602F9B557CC449CD7
:107A90006A640E5483837D0F89801F795B46B23FF1
:107AA00011F5E992DC10A5EC96DC0210C5FE853AD2
:107AB000C18469E98D8EC9596912D93B15A85B66E5
:107AC000DDC7DD358BE2A157343D8EB6F0FB7A6A17
:107AD00095E2E4C193164088828EA6B5B89EEBD29B
:107AE000E39B1C0B9F53B29ED3DC7EB1650BE62655
:107AF0001A32816EA8CE2B3C947477A4C8E1866DAF
:107B000056CC985648EE83A1C76B1F16E0D133D8E8
:107B100091906E22FB5BBB960D6E29A8C08806BBB8
:107B20009207F53DD533B77A93F774C6911ECCB959
:107B30004896304673945B4B7204EA9AE85549EDD7
:107B4000E032BE9741CD0EA7CC03843159471CA427
:107B500011EDD1AB016FEC13572914B084F5D9BEE8
:107B6000C6D8B6F6835B7402659B010BFC6BD38FA2
:107B7000AAF81787EAF54370C723E68CEFD0D03F09
:107B80000D8A12AB6108D85DDC04616DFC0C92704B
:107B900063690D04E160C7C966DA76405FA4B46A20
:107BA00079720F2839FFE76BF28F9384FA758FE3B0
:107BB000B688A3DC02A55EDF9CD2CC727EE8831679
:107BC00077C8809BE214B97F1CD9AC7F152CF18556
:107BD000F05CB403B989A52C393A59530B15C67416
:107BE00026370E9A17A3DBB5AB0742962A16A8D7FD
:107BF00081C72760183C37700B8CF79FF6CBF35E7C
:107C00008F70F74E8F815CBB973FCB174A1DC133F6
:107C1000EBE19B7AED4E15698FBEB1943148FC8F34
:107C2000AB295112946B03CB1AFD61D1AE0D5D30BF
:107C3000E8BB666D443A57D35CCC93E5FA40BAEDA5
:107C40007128F1A4D405DCBDA9D6025618A6804639
:107C5000404DDD7B8B482C82588B7D683588F9F54B
:107C60000944D97127EDDEF1CA2E4D2AD706EC94CE
:107C700061AAD967061D1212FC8EA5E42AAEB1E0F6
:107C800021CD950FCF214F80FA82C7F32466C1150D
:107C90006D20B137FC2BE129CE02389343A301803C
:107CA000126174317869F8066390A774B114E21414
:107CB0009B9DDC9ABC3F916A4C560E66B0EEAE9925
:107CC0001F7BC132275AEF01A96F4636B9BB47D295
:107CD0007396430B82722CC1D83D1F809743A08CB2
:107CE000B5EDAA3643DD86F8C39A0B66911F86E090
:107CF00090A52E2D18198C270FE6E24F0755F94E47
:107D0000238F6EFA2ADA110AE86780C9B758759787
:107D10003B0E112EB2314B8B0E2C083F00A24A7B3A
:107D20005BC07D02F605F4B86640046A121AD6E715
:107D30000DE78463865E382280444951DB76BA4B76
:107D40003024141B7A78000F7CF97F1EB9942ADE48
:107D5000DC7DDA4829566F597A82274B811775A541
:107D6000D0C1CDA786DCE9811B644F4D0A4C21A30D
:107D70005036EDBA5E48914D44F0A811BF5FD9EC82
:107D8000A5374E02BA8A208EE8DBA272AEB5E42B8C
:107D90008ABA439523738914F32BB78158764038F8
:107DA000375A4E5F274530A12A8EFF40C5B603A73C
:107DB000A98DAAD19C955CAB89DA527C5327D764F4
:107DC0006843479DD11280FFE0A8E38CD62863DF8B
:107DD000BCE8A2EDBEA2439F1AE0945D4BDC1A11F1
:107DE000AECF2EBDBA8CBE023EC2BC1F9E3833E859
:107DF000398F0D6DE6B9A7194DC3A6EF985D657172
:107E0000AB0B784D589BE62609837A0429C665A5F5
:107E100096162566722D58DA3DD3E8E3A602A3BB79
:107E20007DA41C44185CE7060E9A62EC507B6F0838
:107E30007C3FC9FA7B0EF5A4BB6563C1BBEE2DAEDA
:107E4000BEF9188EADA293C5FD9E7415169FA2743F
:107E50002B03046B69DFC87D5FADB14AEEB45A5E97
:107E60006C0C15903A03B070623A475416424A8A35
:107E70002FAD987F2EFA0130952B8295C7F2AF7700
:107E8000AB12AB3BF4FD559181FC272A8FF40174B2
:107E9000B0B1ABD041D0F17289B4E78D2B52B76D40
:107EA000A74899345CE551024BD450C77481D58101
:107EB00060D8F5806AC45C03D9FDBED6B2F3CA4768
:107EC00008A757010494869C76C388D37A4E08CBC2
:107ED0006672B8C7B43DDE3862E4DE2FCFCFF5411D
:107EE0002E0BCFD8B64908CF64B65BE9F562F295A0
:107EF00087A16635921EADD86B3975F16F35670B6A
:107F0000BCA6F22BED8788BE348EB8C8D4491B5D61
:107F1000D92D4E36E6A8EA52E8043884EE9AAD1A16
:107F2000D49CBBF40AA00ED56C2F0ED8AF47E1F954
:107F300003FD3C1F67782F5BA85276345A73A7273E
:107F40006EAB48BD3489E5EDE45CAF053280087363
:107F5000726B71DCD9267C8A058A6EAFB73F7AEDE9
:107F60000C2CB8AE1E92E5CA5F65941E7FFBFFF92C
:107F7000032F993C243AC74CDBB9BF0DA36040F9ED
:107F8000FDB120BE3D295BC2362837A8593760981D
:107F9000C0C048F86807B6B0C552D83A7F874424B5
:107FA0003A64A0CE7E52A9DCF5862A22F8FB3E95E3
:107FB000CE12F6338A57C485720A6A51FF73E1956F
:107FC000CD6425745999C16AF00578533ED39B9EC0
:107FD000172F80BC9147DDA2F85A375586315822B9
:107FE00055DB242CF097446503A57CAD9D4FA95D1E
:107FF00023313953F9A8446258486568AD97A0BA4F
:10800000E47003EC636CE8D7CF0F0396956408A483
:10801000923FEC2D4A908E7063E02ACCC61C4A56E3
:1080200023412CC8C0DC9B772037C6A8291B35F814
:10803000856AFF4CEF05F3B9210334FD6BF5B958A0
:10804000BC91E62EAE26A8831BEC0D65B6903E5083
:10805000AFFD8AD99496C077E7F847A3E8FC3620AD
:10806000B9BCE9E8E7021F98AB56623D58FDB1B6CE
:10807000C8763B42CE3555E7F0116ED04671318758
:10808000825C95365D5BFA939A8AAA26AAA0622240
:1080900001131CA4C845B2AD7EE1DB44F1B64A55DC
:1080A000C395FABEF1B60F686541F047A5D4DA91E1
:1080B000CE8ACF043CEBC44DAA1BA89F707738F83A
:1080C000D023BAF211F11E72D2BBFDE235D81612DE
:1080D00046E4348CD84DBD3F6865C3DE5AB0F4E940
:1080E000435C5BD517E0B3BED1BAE5742D669BC780
:1080F00087BF4BEEE31E3AF5F864D82195AFD5372C
:10810000A7385B012BDCD9985F29AA8C376C0AD77A
:108110003F6FF2430B2CCBFCBB40D9E177CFAC4592
:10812000176836ED84C9DDF4A9E68645E2200A3EEB
:108130006CFBC67195BE3FD3BED4F3C4B624D966DA
:10814000C2555A9CCEBBD4740EB1A5ACA9ACE50601
:10815000701033C30541E8FD703AC0FA7F6F603696
:10816000E9D1F41860DCC198FD81CCFC9AB14C15C2
:10817000FA5219C904B648AA988CE17915882235B3
:10818000CA2F4DD19605FBA8EBA461D6803ED1A79E
:108190003D44ED4920A31F59991586D65626AEDFDA
:1081A000BE049A19ACBDCE01F7E0B65A0A82102E71
:1081B000F8E0109773C575CAB002D6DCB0AFA2F371
:1081C0001BB97359BE6718A49ACBB5B9FC6B19A13A
:1081D00034C619AABD400A6C13D39BB66BD5E7D43D
:1081E00071797D501669062BE12984286585A6DF03
:1081F0009510D3F9CC3429DD3854A62D6A4036CBFE
:108200004ECFA70018EDEDC46541FF8AEDC33C9940
:108210004D66C459BAE5E5AF494E9E0B38616D67AE
:10822000ADD991A4B1A3910AA86E431DB9613F1BBA
:10823000FB5786D116AD8A850686F83B2DB397424B
:10824000E975E93FC4EAD17B76B770506EDAE99CF4
:10825000EAC4DC8ADCD31A7FCDBC538712CD28F761
:10826000D3A89C9C5119D3A01A0D2AA3EEC7F75F7F
:10827000D2AAD71C38BAAF24511B0842E3C9E01177
:108280005D25EC70949FEB1E7A412B477AA2AE7568
:10829000E64CB6F1E86DC68211A461A0C49ACE4A3C
:1082A000C9F87805CAD46A042E26BFB97252165F7F
:1082B000D8AF9115B01A006AAE5C229A81BD2D9894
:1082C000495445D5B6C7E8EE8A4E243215ED6E788E
:1082D00036096109052047D8879E1F2697389D8F4C
:1082E0003A9D7494A23D79C4D2550F2C14223615B0
:1082F00043D804CDFEC6914CE682139E1FE1D39C69
:108300001DFE392FDEEB76714527AD989BF0AD3819
:10831000CF63B9969ADF98997DCB7E5FA4590261AD
:1083200081248A6329C3CDF3E7CFFE696DBD4BEE8F
:108330004DA134AE6A36D028392CF9E51BF65D9094
:10834000D6450D170A360A5932A1955C171F3859C0
:1083500097A61E02829ADAC6F0CE73267085DA5886
:108360008A247E7DD34A7EF29DE4D9762405953E0B
:1083700084AE39416A0FE9A796D4C90D72D1BE65A2
:10838000B809A927E91F3E8CCD4E8544080677DF42
:108390005D7CAFA8E69BEA1E9CFE28F19352988B69
:1083A0009138DDC44359C315513CA9C34420A933B6
:1083B0006BB1DBF15499F701E2C9D4224E89D1DCCB
:1083C0005DCA5ED2843AB4B8DD7B3BFE94F32A35B5
:1083D000269A390ED72A03726693A4809D0C53D82F
:1083E000DD243791CDAE632150DD8C1FD2FFF24FDB
:1083F0004EF24637314C105BF980F5A7B3539EAD72
:108400005AAC68F3BF64251A53A00376697ACA533D
:10841000ACD263FB7B21F4CE5DE886A57C9E78AC74
:10842000F90BAD2DBD9745DA9993D1F5091927CEF2
:1084300039F9F4ABA9E1351D864833B298A1EB2296
:108440007843AB165D2691150DD5B9709187C0AAFA
:1084500058D8FBCD5819601A3CAA07B937FD0EC58C
:10846000E185F7D4583F53404E85A94B211F68172B
:108470007192315EA166F88272D0798C9D4BF69B29
:1084800076248D6713F35F4C0126DFC80DABD2D481
:10849000F844611DD363A9E4AF0B47B29FFC768318
:1084A000771FFE6D141661ABCBDDBFA1C6E376DA94
:1084B000F5CA556BBA3D427B1261558CB1B74D0B75
:1084C00079FAE455ECB7D50F52E6B2B5DF92F3AEC8
:1084D000768317970FD1F1BEF8DB263747F31C746C
:1084E0005059BD95A06671E6C75599BE71E3579185
:1084F00016E789E6FF91E751EDEA2EC47377BB30AA
:10850000C6EC66AC1EB91E57FD20FA29E46D7B9FB0
:108510000912198CD6E5C19FC1CA657104ABA2E1ED
:108520007B31644C370C14AF60739042A99934DEF0
:10853000A89117C585D09F16242FE19AB1EEC56981
:10854000A222BF496B763705C949D1A3A1B9B1F4BD
:108550001892DF952803B29798157ED1B966653ECB
:10856000F96353D33192D56B342E5FBC948316F3E9
:10857000D3980669C026960E7D9DC0E7BD73D1666F
:108580004A3BFB6F2A90C5C488BF0791C546B0AE71
:108590001269CCE02498CEE3FB6EA08127CF3A93FA
:1085A0006D759AE5038C92F6370F87FF8A951E76D4
:1085B000C1431634B3A557A2F027603D11593AD1F3
:1085C00016CD7AFD04F940879EA15EB8B651852686
:1085D00085EDC37CD99EF56040DF9EEF8ECA516168
:1085E000EA5A2E765EDC427715A044E444546A06CB
:1085F0005C7B2400F8E1E2E1C38D0073F7F457617E
:10860000D265E3482E284026F2D17C41540F0A0C53
:10861000D895B4FBABFC39FBF0D810AA9377EC38B3
:108620009EC73D4191A250AA7BF902A5CC4977068D
:10863000D62221AF9362AAB9BF15CA86B9589B1139
:10864000BFBD1C916B8E9DAF10BBB13C2227BA9A67
:10865000497C4CBE769F10A130F7F7D3F50FDA2690
:10866000B57EB197DC094611736FB7CD90AFE1A825
:10867000128682A39931CF4BA07718B5D5F0CED80A
:1086800025CCB7CE4F6F2DCF626A64716269870BBC
:10869000DAEE6E0706F7A81D1E67E9530C34228632
:1086A00029AC14EE2355204BB9EC79A813C93BF93A
:1086B000150E78EBE4765D33A240C5EDA22A0E904C
:1086C000AC6247610F0ED97AEE21EEDF6671F6518A
:1086D0005659119D73707454A4FE57707A31C86056
:1086E000FAC34BD9D31414C56FA0514CEFB0A520D9
:1086F000DFD8F0006863D843EA0214D134F295FC65
:10870000911B76CD341453B55923F624B245B5DA0E
:10871000B1B1E287A68DCD8D3FF8BCA038886B1330
:1087200086B923895A44B25895517E75196FE1E68E
:10873000D71F0B43B4EFCCD4E9F56FE0BCCC4B12A0
:108740004E2FD011F16F4543152DD3188314DF95AB
:10875000809916649D1164EEAB10FC1450BB4E89D9
:10876000CFAAE5077E5717C5C5CFBEC08AC1D5E4DD
:1087700046295FCC4DB1AF63DB488CFAA68C4B9792
:108780000216A09E9B122FD471898E97B2FFB2C1A0
:1087900003AD9E03F7830A89BBE49A7EC258EC912D
:1087A000415F4250DBCB40E81B808B760BEBB17E08
:1087B0003DFBE4080EE422FD37BF6AB1419D71BC68
:1087C00014C419CEAE42FE27AA21B9C6D3973B7274
:1087D00091D35352E746C44A73AEDCD6689927A9B1
:1087E00092AD59828DE8981E9B9345B5B61420BA78
:1087F000833D5F28FC02086EDBB289B07368ABB5BD
:10880000CC5C4103C5005CC4B6A3E67F32A1A6667A
:10881000E6AE9D6196B73C7801A5C431A8056F8787
:10882000DC035F2C6C73FF6C38F2C4A7B64AF1C945
:1088300006AD8EE9E0178E22C7A78B698C6C9989EB
:10884000D8674D35B2852FEA4CABE73EE48351DA69
:108850005283CEE2AE205B70E6A8FD08F18B1E3994
:10886000666B738E75C1A5B805D7CB1278CFD4725D
:1088700031C09A12EF96FEF18B05CC00E918B9874A
:10888000351122060B57D2182C1A30E5FB83D6443B
:10889000A8ACFDAF91AE8F8EFA1A161B768FA3404F
:1088A000B22F981ECA8B8857C7AB8CB8587148C86E
:1088B00095880BDAF604C263E333769D2DF00F2022
:1088C000647415BEEEDF48171F6AA35AF7AECC607A
:1088D000DDA4835F68BA1838AC27BA96BC28785AEA
:1088E00099FF89BFA52172498D9CF4FD41874C4EAB
:1088F00066C0F21DEBFCDDB1EA1E3A0EA3711FFA51
:108900000CF99CE3F505AABA0EC739075BB09F12B4
:1089100061F152E1C574546C77669686FECF22A051
:10892000A57ABAAD22402D0F9CA60701A9B6A19A3F
:108930008B523EA0DD9A3005DF991CB9DA7E26CE37
:10894000B9E4A1B8BF90F2001ACFBC037532CEE1F2
:1089500067052C1124D0510374023CE7DBA467FEA9
:10896000DEA708C56801A53E534798EBCCA669472A
:1089700084D694FB418EA7073A0E5A6AFDCD14F6B1
:10898000C1E2141B2815E71DA10E5CCDD9D4E8ACBB
:108990006C5C431409A159CF61177FD45F818A872A
:1089A0001B45C4F5EFA5ACCDE1A1AB59B742A01F63
:1089B00053692328636BD3A8F5A05A5E397EAA8B2E
:1089C00097364DD2B6BDE0DBAA49921FFAB04230CD
:1089D000DAF116F31A85550B07F341F91B8D3C4C60
:1089E000DDA036047A7E2F45F80052B919CA131C4F
:1089F0006A31F43CE2CCC2A651F1667C54FB2CD225
:108A0000F5F1C9A7AF412293954E2F99E02E2D1372
:108A1000F03526459014A5326C10A2346E2ADE85FE
:108A2000D859DD9D2B4CD8EF21DE68652E77B21C1E
:108A3000564C50BF6788B783462ABD1D42CF22A13E
:108A4000DF918E4411E648B187EDDB360FB9F0C3F4
:108A5000A6F9B0A4FCEF80E018472B35AF8B4C860D
:108A60008C4102CF55F25DBE1659D844F9158E4D92
:108A7000570947A1D28D2DD5ACF9C89C9183B6FA80
:108A8000B95F5A3EEE4D780102567880C0DB092C62
:108A90004E4C1B677350B6BA5C0F59E04D36FA0264
:108AA000431293D0E1A73939DAB4A050C1CA160BEA
:108AB000CEFD308B3714DB0BF1856377669EC58E58
:108AC0007D9B75B2A080FB8F37435801F5C777D0E7
:108AD000CB847543F6211E19BAA4D2F00DD004D56B
:108AE000A3534DADBD7733867053FC40DA19B655AC
:108AF000DA948F0FC06336FA7E087B2E0D55912EC7
:108B0000AA0775F4B5F3D24A08E9A41F1C2F29D28D
:108B1000E50EC5F0662596AC2E13F2748104E98645
:108B2000B65269068584E58FC43BE4021EF95727D7
:108B3000312138FE67B6189EC43AA1F848C23D26D6
:108B40008CAC946BC90FE31F13068626B8DEC85A97
:108B500064724E281E4821B44CC77809EBA5F80270
:108B600081B17C94D6B15CC13C4934FF98F3F84B99
:108B7000DC01469E6398AFD02AB699E8D063359061
:108B8000026E5BAD98E2DE7536FB447F94B601A7BA
:108B9000DF06E9EC4D2AE1D166D4DEDE6A98351DA8
:108BA0001C778249ECED67ADF53A6BC025DD25D821
:108BB000B53D15484881155398C067C0D3A01847E4
:108BC000FF4BAFAA43F9C9C8E14D9280DBBE415DBE
:108BD0005300CEF5C5D4DADEC2F8DA959E09588F77
:108BE000B3FC322410E2DD9B2560602F62E4737BCE
:108BF0000083E7298983A0C3C9D8EAE0959F81CB88
:108C000078A23F4FE1C18407ADFE03C3FBAB3A4DF1
:108C1000B14A8722407260325A3D5367B2FF21AF9A
:108C2000745616ADDB38FFAA5DDC879DF21D84A368
:108C30006C5E94FC6323F43EBBFA61E50038ED8A78
:108C40002998F426EF3233E0148698972E9BE87E1D
:108C5000FB017E431A5B4021EC5878A1425A9A2EC0
:108C6000BF412D9897617B135BC85BEADCF478BD4C
:108C7000BEE3D585291EB7D8A1FB5F201C27C18B79
:108C8000ECB72E7863684AFE8FD2F353725B276984
:108C9000D56BDC4F6F7CD52F277F844D4727CD9731
:108CA0005B447E6EDC95E7A59CE80F53FF3FDB1726
:108CB0002FC6E567EAACEAAC69934B02643441CE57
:108CC000BA4A4B58009DF89111AC527820068A2977
:108CD000F62CA18864FCA837481EBCEAEAA8F64036
:108CE000A799393564DB9C240248E94C6F40CB1EC0
:108CF000EB979F381983FBBAA80AAC6A46A1FEDB42
:108D00001021651F78A7D690D521443A51D46BB86D
:108D10008552A1BA1DFFD439C883AEFB2AEFCFC755
:108D2000E45A68D43C6443765509BCB350168FB6F8
:108D3000325C65093F4D925B534F9439FE4AA4AAB9
:108D4000D1447C022DC0B794D9292365C54891D35D
:108D50009F5810F49AC3ECF5566CA1800EAF5724BF
:108D6000541CAB2F64EFA13E0D08E65628C20AF949
:108D70005D39298B4E523E816BE74A28E1CC52FF88
:108D8000DC8957904AB89F1ECC1C1DEABEEA45D626
:108D90004315DEE21E138FACDC39C18CB7FC62DCFC
:108DA000EACDC1BEEF72CAE083768AB2CDC7FE07B4
:108DB00019124ECCC83A952DEA5AFBAD98BE96BD15
:108DC00022ED5E72563ACA245E2F8905A5216048BD
:108DD0004C22BB89E0B49F8202A956B1DD081D4434
:108DE000466D6E5F48B2AFA93ADD3FC126D57C6AB9
:108DF0006301F80D4A335D476D2058303A05BCCD0C
:108E0000E0B8A1E1B74B1495AF07E6E757C7047088
:108E100090718E935D77928527293852E9A94D8C00
:108E20009EE7AA8AC77FEFF16653F634BE0B263859
:108E30006B04FB39153BCB95D5B283F9C25B036755
:108E40000CE7D2E559FC2E2F7C3EA6E4E26EEA3315
:108E5000A5B5DCB39D3207AC0A1D5E18D131D71B16
:108E600034A3557C4F0F061069D1DE066AB7FF396F
:108E70002F04E1F30AC3026A6A6062BB3E078E28D0
:108E8000136FDF742E72B17B69CCE62FC03A712C60
:108E900068022CFF7390ABDBA85F68D7FEECF6602E
:108EA00018FF11E190D999B9CAB62040750E4AFE53
:108EB000EF2B8D5F0186E4F55A266B012619E267D8
:108EC00097ECBA98EF0905C91FFE179D9C827C6537
:108ED0007FB8F4C8080AB6473B7776B7290A4ACD67
:108EE000EBF8E3A91A7C4A77EA63C84920F6599758
:108EF0009685376166EEFDED4A409870F8B1D7DF90
:108F000008AA3D683FECFC8A814967E3AF799A7F04
:108F1000D86987F6382D4E39E6DB7DBEA2F8974139
:108F20004D73FA240AB47B50074A420750AE4029D9
:108F3000FEFDE891C33D777AC3690D7C7C2A11F070
:108F4000138A2B78F57E541A076635AACD6F030F66
:108F5000B83753883A16F602DC8B2E8B7DAB6B93B9
:108F600087564D2F9FA967CAAFA228C4B094E07A54
:108F7000D9134B7C6F6F7CAAF297ECA1CCD15D2703
:108F80004FD06CB42C4FBDE625DC69C41079F09A43
:108F900059B2843A389460645ACC63818AE5E88097
:108FA00042DCC56A661228055AA52AC72B810B8D9B
:108FB0001637AFBE6AC43ABAA8FDE6DE6D2082F964
:108FC0009E860A36C0F9E98881D86AEA11BB5084C6
:108FD0004A76612045C8EF81026DD6CEBB27E2F606
:108FE000C16F7D4E181AB21E87E2E9243B5ECD8424
:108FF0007ACBD7CA6D62C252EAB065734B363CBEBB
:109000005D417F9840AFBB7D1B4BD1B58AEB3DA046
:109010007D1420405239F2FC1548FC3D7A125093E1
:109020008F91A886A9BC182F38A1601C1C4FF13362
:1090300047BC066CB405486FD30BB7B45D9BC2C088
:10904000661783101776797738F820DFC9C31E2991
:10905000560314E095871464F2CEE2351991FF3679
:109060007538701953CFBA175E377A73EF3F97325E
:10907000D0321DEBC78C70ED4E36193D0F38A40F62
:10908000A46FA296FA4983E5B8B241A29BD00B5DCA
:109090002299242523D4A434E43328AB3AA4EDD177
:1090A00055960858E84D314047FB9066A53953C2A4
:1090B0007B309A056567DA593B997296357B75F472
:1090C000EB1681F436D57ED02ACC4A24F5F3800203
:1090D0003E8CBEF1B92B325EDD02B0EBFEB655031D
:1090E000EC5C741121F2262A04DDD86A7D00E22EA0
:1090F000FD73FAA11D5A68ED5130562DE34953C155
:10910000AE5957021305DEF441BE3A30E90C8539F9
:109110008A1DB03805048EF34C2C196CCA66A87AE7
:1091200088E78E75DABA7C9B166D86513C7E53BB00
:109130005A01970AE353D80F6EAA9EEED288C54A09
:10914000717B72736C769CE0940A5CB2F3F7D7DCA7
:1091500073DA937E2E34DB1F71183E417E6024202B
:10916000A8E54B2678CD53AE2DF31E019A5966E043
:109170004AFE93A259C67EC8C76CB0B834549074E6
:1091800006ECD82A18AAA615CB568274B4712C41C5
:109190003F6AB6F3974A79E1C5A3319EEACD50D034
:1091A00006516F8C456A796860AE77CEED65EC65E7
:1091B000264217920AA4BC3772E96D4C0F34B7826D
:1091C00009273C72AA8551A3B7A6219164BD9930A5
:1091D000C5CC7D443D6E33D0922D9B2233502DED76
:1091E000E5066AE4E7032A109ECC87F116051E21E6
:1091F0009C7C8773EA89AECC88368832DB1FED2DE4
:10920000D5B74133109C9B708026F446447D543979
:10921000628B18D59C6F3FE269B5B907B4E44B3156
:10922000FA79BA9ACCED4A4936DA564EAE6B795194
:10923000209CE1C6D6B92F7B170B7B744BA3019CF6
:109240002E172C0DF19D1E438665FBBD8F251F112A
:10925000A3383D42A4195E143002BA3F14B1DF3581
:10926000F68594D03071375ABECED433D15BEB9EA5
:10927000D6C8260B827073BD548672590C6B1606C5
:10928000F54B7541F452F69E9FBC46B1308CC16CD3
:10929000A5E4A32332D29A324F381AB247F98F6825
:1092A00064FB3FF105BD0C939E6C79AB72FEC82345
:1092B000DBB0A72D517D478F5C1004819CE895A7FA
:1092C00037FB4E054FB6B91CDD21D63570FCF237A1
:1092D0001D78AF9DF7E73CBFA023B5CDF79645724B
:1092E00098BF9937B710A99CE0F2C36E83BE03AB59
:1092F000B7D1B210FADEA2776B3BFB55A0F6831F05
:10930000FC89AA8993BF35599F211873B4F4C85AB0
:109310004DF6EE735F4A564E02E44AAD7D3610BB01
:10932000717502027F7B37CC6E021737B85A59C36A
:109330007E0004E8D6FB0D7F9C3CDFCB6B1B7818CE
:10934000FE210AB00067141EE4DB6D0B991736830B
:10935000EA42AE9B555C1A574550871D20578EB385
:10936000FB4C4D80955E2DAC969CF0787F58574213
:109370003126EEBF202AA3870224E61C3231B6BC78
:10938000C6929A1A151AB27C82A7D25BBAFC2E6DCD
:1093900098A4EB9C45B14A70FBBF4334B8F2BA0ABB
:1093A0000DC334B41C459F407B95F6B111801A0E55
:1093B000BF3F012D357B21A9C7F25E3B896C32444A
:1093C0007E1160283ECDBA739C40B1596BAC2C968F
:1093D000EBEC20FF99D672AE85EE4BF75516F5B63D
:1093E000C3147A0EA76D44A644FF574B0D132FCD1F
:1093F0009649BD8FE89E175946579CE9E1A72F096A
:109400009E4504159FB54892105A6147F99AD67146
:10941000B849ED6B754AF82A5A4F69375CEC5C64C1
:10942000F13F1DAB9802DE197C97DB53C931D9D7C8
:109430009CD3A799CF3357121D951B911F0653FD3F
:10944000DCB01D38CA121ECFC2833901426DAC6A2E
:1094500025B3AA35B334A210371557F29EC1E0895F
:10946000D15BBA86C13B923FDB2CD0A26BF13AC2F2
:10947000AE0E10AC8D87CA2F5EE6402CC27AB6992C
:10948000CE14F088FF2D9668F97625073E3B5AC921
:1094900032C840CEEE65A43D316AE92211F1411790
:1094A000BF8021DA9D2CA2E8CA6F7E3A8ED8DAC33B
:1094B000F54B34788A75F28ABB8D81E0F9C718A81C
:1094C00022F8406394AFD818F1808D9C81207854A5
:1094D00020C5EB35CB3BC89A1C7BE6192B12549860
:1094E000B34918096C2AEB7FA3559D0964402ED718
:1094F00056ADA9ABC265F69B13AE2E30D5476BFFB8
:10950000EA1CA842EE20609CFFEEE2D7B04A1C7C29
:109510008E691F64C9E5ED66FDB9DF53F931F2FFCD
:10952000B707C15980993B1C4C01307D101FDC727C
:10953000DDB8D2D6D46F4C5C517B84959B910BF6F1
:1095400011399FBD9485FF03D4CA9B901446033103
:109550004D9197B21756B80BF84197E841A933F9E6
:109560009A2B2BED1E3AB3B9FB819F8137C5A9EC2D
:109570009946F5D99D8EE85E9DA9E4125751E8877A
:10958000A10307CE518C160982E7C291FEA66E4454
:10959000A79E8BC4470ABB503A16CE7B446E2FDB86
:1095A000D87A4D8CC5FF302E7A8E581EDDF300D14F
:1095B000A468E2818AE25B3B6862FCA52832E2F79C
:1095C000285EADE6F591ED1F7F96C28A954C50ABB3
:1095D00022FA98FB05C7E7038073904E1537A180E8
:1095E00099463FB2EA53AE8C1D33A72F70135DA589
:1095F0002232DFFCF4F56CEA794C76A1EC25030FFE
:10960000546E7134DFA578BF7F50958D6C395CC482
:1096100048158DB958007095F7CE2C385D37F29DFE
:10962000640C08D31D3B2D824FEE82656FDFE3890A
:10963000C5281D3B389623FBB03362A2AF86D355B5
:1096400087C7C84093FB1F290CF8F4E7F0EF387682
:109650006FE53B2CB7BA4774DD1CBC08CAE2B622E2
:10966000A85FD85AEA0A9F5454DBA8C7882F2D5503
:10967000FE3793CC5AE5F071EAFC6C93B895F6D8B6
:10968000AB36E6AE6DEB07B21B559E0808AE2671F1
:10969000F2B5741998EE87D3625BE74B624EBDE674
:1096A0006D306C07ACDB2253B3C2F0FE68E27AED9A
:1096B0001EDE54B578264AE961A9D19C3F631C9D02
:1096C000233E3C9D0A8CBABFBA05730CAE1F8AD4E8
:1096D000A2B361CA664C24DEBEB50A0503F85E3F3C
:1096E00067232CC83DE4D06AC314CC08EB56CF39AD
:1096F00007BBAA4DA2B288FB3FAE7D1D3931E5EA1A
:10970000A416A5F970609CBAE7106F95DDD4C1CBA3
:1097100000C81AF502CA6527AF7145BA1D62C9AE05
:10972000A2D2ACD4B3BC840AA37D07866648535842
:109730006DF58CFAD2CFC6FD5A5011062048B614EA
:1097400056041E51F4F6B881BD15706716AD0BC3F3
:10975000EE9753CB0AF78325B18EAA42194DD7BE97
:10976000F24FC35C36528F95CDF87A07390A352A05
:1097700003E4B1559F44F80F6775E13A840B39E073
:10978000D8CF0586B3A8745F56AEF5D03766A484EB
:10979000FADBBAE8C6E1B02E8D397FE6DAA0C7FA67
:1097A000928530E13F73FFC237A1B35CDE67D2D44C
:1097B0007EBAE4BBB1E5BE1F06B467F9B51BA79539
:1097C0003CC142C56605307086D2E7D2C238F07718
:1097D0005A617116C83E1730A22923F2318415A4AC
:1097E000412EE78123ABA4A2F6FDE466F5686D7C0B
:1097F000E078601F3300D8DA7DD7E00F1DDABA4B6E
:109800004A378811A7DA1962C80844D8A714D3DAEE
:10981000C954F68466D0AC81CED83891FC98772DA7
:1098200028AC41D10C2A36FB84159148DE387EE7FE
:1098300064E1BE51687CF269865BFF1F7141D75DB0
:109840007346FA500832DACCE41C03CA4D1938A327
:109850006F6DF31841031E0AF6BAC1E06E29AF8599
:10986000F03AC3CD222DB3D7E1E6C2E4DD431AB806
:10987000FBF3A64B9AA49496C416426A5828F72E76
:109880004CCE6B16495AAB2351422ABDF416E60F53
:109890008F061897E0C4FC404A88E638FB24ACBE2B
:1098A000FA62533A1F18BF1B09E5C14400CBB3BA93
:1098B0000E63CB7925DAF12ED9E701B5DF360B89B6
:1098C0002DD63ABB3FC2691DB2434560EB2EBF2483
:1098D000FEF546856830547DA9C74909F1001FA6E9
:1098E00098BA6C897CFFDCDD42E9BBF32F3C0B2A84
:1098F000225FE1A6C751B1149B530B5C79CD019057
:109900006896E2DC0950F5A4DCAB2287B1FFA39C8A
:1099100004C7748319D2130A4C58ECD167587B845E
:10992000590A0554C8B1C5C2DA7AAFCE3C1D5FCE24
:109930009AADF3B3016B2E937B3FCF7A9BB8EFDBED
:10994000FC1A981C1A477E29BC25C3B9D6E196EDAE
:10995000C4A84B9661B4DDF5C2B068887E5AA1BA3E
:109960008BBF7DC58F77849CEB1A36DE9B7E497951
:10997000AD24914D82B48505F61B3676D8AED5EC74
:109980005D84E9C9BCC8A8BD8F1C1BA15E0D63D452
:10999000D1DF3F474CE512CBF72FCDF7B9D7255B89
:1099A000E41990C0CD82EB40D114ADAD5C9A6D63EB
:1099B0002BD1724201E5152A7C66D9851C2458D822
:1099C000431D7A76F7D129CC1CB144324AFF076394
:1099D000ACB449868730A6312CACD29CEAB9BA74B3
:1099E000B673A23378F46FCD45105A973D762DF7B4
:1099F000BE79F01B80A7EBA0DEFC94BC5295DCDFA7
:109A00004C9275D9FBE6FFE1189070F2845B729E70
:109A1000637618B0B656E1C344DAEC9541B0367BB4
:109A2000DA57F0166D9ABB1F877DC7940659C63763
:109A3000FD2694038211DCE11E0D272261AA136723
:109A4000C8DE6C80A99F5DA67B3F1249C794DCCF1E
:109A5000D6492A735019A78D4947FA44538F031BDF
:109A6000F376253968AF786BD8B66B53E3B7E9B4B2
:109A7000D82EB2231998AA0FFCB10B6D0A78F414F2
:109A8000D2C445C4169A9E679E6300326839BCCE24
:109A9000E6262D880D6B79F244038D201175C5E8FB
:109AA0004AEADC92DAAE0ABD3A5AA11B832C56FE72
:109AB000AA17D03CD9EEBEDB217453C6AABEAE268F
:109AC0002F78618DAE3B861BD2A88EBD31A6642F48
:109AD0006773060C95E73A766197B879E1C728CFA6
:109AE000617A74382BDF5C585AB9FAAB13F9386ACB
:109AF000658BA213E6B178A9E60981902254B2AE33
:109B000047CFC94D71A33293983B2FA71C6E38667F
:109B1000C989804B652CC49EC1B9C548853CFE48A7
:109B200008D05227FD4A4EAA0304050A08060BFF77
:109B30000209070D010C00FF202569202569202559
:109B4000692D256900202025633A25690020202001
:109B5000205F5F7C002C00610044697370206F6699
:109B6000660D0A00555345520046004700424547DE
:109B7000494E0052414400442E4D59005052474D29
:109B800000555345522020200066202000672020E9
:109B900000424547494E20202020200052414420C9
:109BA000202000442E4D592020200043202020005A
:109BB000081C242C4448586C7405000000FFFFFF6B
:109BC000FF4D000000FFFFFFFF0F000000F4010049
:109BD00000040103010201010411040F041704161B
:109BE0000118010000819B0000899B00008D9B00F3
:109BF00000919B00006B9B00009C9B0000A39B00BE
:109C000000AB9B00007C9B00000502050804080BCC
:109C100008040405010504090809040608070206EA
:109C2000020402060106040701030803040C080DE0
:109C3000020C0203020C010C040D010D080D0408B6
:109C400002080807080202070408010804090209BB
:109C5000010A080B020A0201080A010A040B0102A8
:109C6000080204100811021002110810011004115A
:109C700001120212011302130812080F0812041332
:109C8000011304140214011502150814081708140E
:109C900004150115041702170119081A02190216F2
:109CA00002190119041A01160816041B021B081ACE
:109CB0000818021A041B011B04180818040B0420BE
:109CC0002020202020202020200000000003000071
:109CD00000649B0000699B00006B9B00006D9B0073
:109CE000006B9B0000739B0000779B0000C75E0029
:059CF000007C9B000058
:00000001FF
